:10000000A2C20000D1C20000CFC20000CDC20000D9
:10001000CBC20000C9C20000C7C20000C5C20000B8
:10002000C3C20000C1C20000BFC20000BDC20000C8
:10003000BBC20000B9C20000B7C20000B5C20000D8
:10004000B3C200000C94D924AFC20000ADC20000BE
:100050000C949530A9C20000A7C200000C9485231F
:10006000A3C200000C94A8210C947F219DC2000023
:100070009BC2000099C2000097C2000095C2000018
:100080000C94AC2491C200008FC200008DC200000D
:100090008BC2000089C2000087C2000085C2000038
:1000A00083C2000081C200000C947F247DC2000046
:1000B0007BC2000079C2000077C200000C94522479
:1000C00073C2000071C200006FC200006DC2000068
:1000D0006BC2000069C2000067C2000065C2000078
:1000E00063C20000E002ED02F602FF020C031503FA
:1000F000B106B106B106B106B10622032F033C03D7
:10010000B106490352035B03680371037A03830357
:100110008C039503B1069E03A703B003B106B10695
:10012000B106B903C203CB03B106B106D403E103A0
:10013000B106B106B106EE03FB030804B1061504CF
:100140001E042704B106B106B10630043904420486
:10015000B1064F045C046904B106B106B106760429
:1001600083049004B1069D04AA04B704B106B10645
:10017000B106C404D104DE04B106EB04F404FD04AA
:10018000B106B106B106B106B106B106B106B106B7
:10019000B106B106B106B106B106B106B106B106A7
:1001A000B106B106B106B106B106B106B106210528
:1001B0002A053305B1063C0545054E05B106B106D5
:1001C000B106570564057105B1067E058B059805D6
:1001D000B106B106B106A505B205BF05B106CC054D
:1001E000D505DE05B106B106B106E705F005F9054E
:1001F000B106B106B106B106B106B106B106B10647
:10020000B106B106B10606050F051805B106B1061F
:10021000B106B106B106B106B106B106B106B10626
:10022000B106B106B106B106B106B106B106B10616
:10023000B106B106B106B106B106B106B106B10606
:10024000B106B106B106B106B106B106B106B106F6
:10025000B106B106B106B106B106B106B106B106E6
:10026000B106B106B106B106B106B106B106B106D6
:10027000B106B106B10602060B061806B106250640
:100280002E063B06B106B106B106480651065E06CB
:10029000B1066B0674068106B106B106B1068E067C
:1002A0009706A406FF080409090913091D09960900
:1002B00027092F09370941094B09550964096E09B6
:1002C0009609780982098C09771F7A1F691F6D1FAB
:1002D000731FB11F7E1F821F881F8C1F901F961FC8
:1002E0009A1F9E1FB11FA41FA81FAC1F4E414E494D
:1002F0004E495459494E46CDCCCC3D0AD7233C17E4
:10030000B7D13877CC2B329595E6241FB14F0A0030
:100310000020410000C84200401C4620BCBE4CCA20
:100320001B0E5AAEC59D7400407A10F35A00A0729D
:100330004E18090010A5D4E80000E8764817000020
:10034000E40B54020000CA9A3B000000E1F50500EE
:100350000080969800000040420F000000A0860137
:10036000000000102700000000E803000000006407
:1003700000000000000A0000000000010000000072
:10038000002C76D888DC674F0823DFC1DFAE59E147
:10039000B1B796E5E3E453C63AE651997696E8E6B6
:1003A000C28426EB898C9B62ED407C6FFCEFBC9C89
:1003B0009F40F2BAA56FA5F490055A2AF75C936B9B
:1003C0006CF9676DC11BFCE0E40D47FEF520E6B556
:1003D00000D0ED902E0300943577050080841E0830
:1003E0000000204E0A000000C80C333333330F984E
:1003F0006E12831141EF8D2114893BE65516CFFE15
:10040000E6DB18D1844B381BF77C1D901DA4BBE4A0
:1004100024203284725E228100C9F124ECA1E53DE2
:100420002700002100240027002A002D003000337F
:100430000001010000040107010A0101021020204F
:100440000808102040102040800201020108040228
:10045000010102040810204080804020100804029E
:1004600001800402018040201008040201080402F7
:1004700001010204081020408001020408102040FD
:100480008005050505070508080808020202020A9A
:100490000A08080404040401010101010101010327
:1004A00003030303030303040707070C0C0C0C0CE2
:1004B0000C0C0C0202020206060606060606060BD5
:1004C0000B0B0B0B0B0B0B00000A0B02090C0D0E98
:1004D0000807030401000000000000000000000005
:1004E000000000000000000000000000000000000C
:1004F00000000012111000000000000000000000C9
:1005000000000000000000000000000000000022C9
:1005100000250028002B002E0031003400020100CD
:1005200000050108010B010000200023002600291E
:10053000002C002F00320000010000030106010919
:1005400001009C47984711241FBECFEFD1E2DEBFC8
:10055000CDBF00E00CBF17E0A0E0B2E0E6E3F3EAB5
:1005600000E00BBF02C007900D92A434B107D9F789
:100570002CE0A4E4B7E001C01D92AF3EB207E1F762
:1005800012E0C2EAD2E000E006C021970109802F04
:10059000FE010E947E50C13AD10780E00807A9F70A
:1005A0000E94283D0C948A512BCD603E710508F0C5
:1005B000D8C3FB018827EE58FF4F8F4F0C947E5015
:1005C00081E090E0A0E0B0E0809358079093590755
:1005D000A0935A07B0935B07089510925C0710929E
:1005E0005D0710925E0710925F07089510926007F2
:1005F000109261071092620710926307089581E0DC
:1006000090E0A0E0B0E08093640790936507A0932A
:100610006607B093670708951092680710926907FC
:1006200010926A0710926B07089583E090E0A0E0B3
:10063000B0E080936C0790936D07A0936E07B09322
:100640006F07089588E790E0A0E0B0E0809384070A
:1006500090938507A0938607B0938707089588E74E
:1006600090E0A0E0B0E08093880790938907A09382
:100670008A07B0938B07089588E790E0A0E0B0E088
:1006800080938C0790938D07A0938E07B0938F076C
:100690000895109294071092950710929607109261
:1006A00097070895109298071092990710929A0749
:1006B00010929B07089581E090E0A0E0B0E0809365
:1006C0009C0790939D07A0939E07B0939F07089562
:1006D0001092A0071092A1071092A2071092A307F0
:1006E00008951092A4071092A5071092A6071092E1
:1006F000A70708951092A8071092A9071092AA07B9
:100700001092AB0708951092AC071092AD071092AB
:10071000AE071092AF0708951092B0071092B1077C
:100720001092B2071092B30708951092B407109276
:10073000B5071092B6071092B70708951092BC073C
:100740001092BD071092BE071092BF070895109235
:10075000C0071092C1071092C2071092C3070895F4
:100760001092C4071092C5071092C6071092C707CF
:1007700008951092D4071092D5071092D6071092C0
:10078000D70708951092D8071092D9071092DA0768
:100790001092DB0708951092DC071092DD0710928B
:1007A000DE071092DF07089581E090E0A0E0B0E05E
:1007B0008093E8079093E907A093EA07B093EB07CB
:1007C000089581E090E0A0E0B0E08093EC07909382
:1007D000ED07A093EE07B093EF0708958CE291E048
:1007E000A0E0B0E08093FC079093FD07A093FE0784
:1007F000B093FF0708958CE291E0A0E0B0E0809311
:10080000000890930108A0930208B093030808958C
:100810008CE291E0A0E0B0E080930408909305089A
:10082000A0930608B0930708089510920C08109240
:100830000D0810920E0810920F08089510921008DB
:100840001092110810921208109213080895109235
:10085000140810921508109216081092170808959F
:10086000109224081092250810922608109227084A
:100870000895109228081092290810922A081092C0
:100880002B08089581E090E0A0E0B0E080932C0870
:1008900090932D08A0932E08B0932F08089585E01B
:1008A00090E0A0E0B0E08093340890933508A093E6
:1008B0003608B0933708089585E090E0A0E0B0E0F6
:1008C0008093380890933908A0933A08B0933B0876
:1008D000089589E190E0A0E0B0E080933C08909317
:1008E0003D08A0933E08B0933F08089582E390E04E
:1008F000A0E0B0E080934C0890934D08A0934E0880
:10090000B0934F08089582E390E0A0E0B0E08093B8
:10091000500890935108A0935208B093530808953B
:1009200082E390E0A0E0B0E08093540890935508F3
:10093000A0935608B0935708089582E390E0A0E092
:10094000B0E080935C0890935D08A0935E08B0933C
:100950005F08089582E390E0A0E0B0E08093600833
:1009600090936108A0936208B0936308089582E3AE
:1009700090E0A0E0B0E08093640890936508A093B5
:100980006608B0936708089580E991E0A0E0B0E0C0
:100990008093740890937508A0937608B0937708B5
:1009A000089580E991E0A0E0B0E08093780890930A
:1009B0007908A0937A08B0937B08089580E991E0C4
:1009C000A0E0B0E080937C0890937D08A0937E081F
:1009D000B0937F08089510928408109285081092B1
:1009E0008608109287080895109288081092890846
:1009F00010928A0810928B08089510928C08109219
:100A00008D0810928E0810928F08089510929C09FC
:100A100010929D0910929E0910929F0908951092BC
:100A2000A0091092A1091092A2091092A309089599
:100A30001092A4091092A5091092A6091092A70974
:100A400008951092EC081092ED081092EE081092A2
:100A5000EF0808951092F0081092F1081092F20831
:100A60001092F30808951092F4081092F50810926D
:100A7000F6081092F70808951092FC081092FD08ED
:100A80001092FE081092FF0808951092000910922B
:100A900001091092020910920309089510920409A5
:100AA000109205091092060910920709089585E031
:100AB00090E0A0E0B0E08093140990931509A09312
:100AC0001609B0931709089585E090E0A0E0B0E022
:100AD0008093180990931909A0931A09B0931B09E0
:100AE000089585E090E0A0E0B0E080931C09909329
:100AF0001D09A0931E09B0931F09089584EB95E189
:100B0000A0E0B0E08093240990932509A0932609E2
:100B1000B0932709089584EB95E1A0E0B0E08093BD
:100B2000280990932909A0932A09B0932B090895C5
:100B300084EB95E1A0E0B0E080932C0990932D091F
:100B4000A0932E09B0932F09089585E090E0A0E0CE
:100B5000B0E080933C0990933D09A0933E09B09387
:100B60003F09089585E090E0A0E0B0E0809340095F
:100B700090934109A0934209B0934309089585E0F9
:100B800090E0A0E0B0E08093440990934509A093E1
:100B90004609B0934709089510924C0910924D09E7
:100BA00010924E0910924F09089510925009109218
:100BB0005109109252091092530908951092540944
:100BC00010925509109256091092570908951092E3
:100BD00064091092650910926609109267090895D8
:100BE000109268091092690910926A0910926B09B3
:100BF000089510926C0910926D0910926E0910926E
:100C00006F09089510927C0A10927D0A10927E0A54
:100C100010927F0A08958CE390E0A0E0B0E080930A
:100C2000800A9093810AA093820AB093830A089560
:100C300081E090E0A0E0B0E08093840A9093850A80
:100C4000A093860AB093870A089510928C0A109296
:100C50008D0A10928E0A10928F0A08958CE390E00C
:100C6000A0E0B0E08093900A9093910AA093920A3A
:100C7000B093930A089581E090E0A0E0B0E0809303
:100C8000940A9093950AA093960AB093970A0895B0
:100C90001092A40A1092A50A1092A60A1092A70A0E
:100CA00008958CE390E0A0E0B0E08093A80A9093D0
:100CB000A90AA093AA0AB093AB0A089581E090E034
:100CC000A0E0B0E08093AC0A9093AD0AA093AE0A86
:100CD000B093AF0A08951092B40A1092B50A109218
:100CE000B60A1092B70A08958CE390E0A0E0B0E055
:100CF0008093B80A9093B90AA093BA0AB093BB0A3A
:100D0000089581E090E0A0E0B0E08093BC0A909369
:100D1000BD0AA093BE0AB093BF0A08951092CC0AF0
:100D20001092CD0A1092CE0A1092CF0A08958CE349
:100D300090E0A0E0B0E08093D00A9093D10AA09315
:100D4000D20AB093D30A089581E090E0A0E0B0E029
:100D50008093D40A9093D50AA093D60AB093D70A69
:100D60000895660F771F660F771FFB01E85AF84F4B
:100D7000108211821282138208950F931F93CF93D2
:100D8000DF938C01C0E0D0E0BE01C8010E941C3698
:100D9000882319F0BE01C80108DC2196C13ED105A7
:100DA00099F7DF91CF911F910F910895EF92FF92E4
:100DB0000F931F93CF93DF9300D01F92CDB7DEB771
:100DC0008B017B01EE0CFF1C622FC70129833A8344
:100DD0004B835C830E940D4F29813A814B815C815A
:100DE000992757FD9A95852F742F632FC701019678
:100DF0000E940D4F0D58110929813A814B815C8168
:100E000003301105A8F4BA01992777FD9095892F31
:100E1000C70144960E940D4F29813A814B815C8124
:100E2000652F772788279927C70145960E940D4F80
:100E300080E090E00F900F900F900F90DF91CF9196
:100E40001F910F91FF90EF9008954F925F926F92D4
:100E50007F928F929F92AF92BF92CF92DF92EF924A
:100E6000FF92CF93DF935B01EB01CC0FDD1FCE012F
:100E70000E94054F482E512C612C712CCE010196F9
:100E80000E94054FC82ED12CE12CF12C8DE8A81A18
:100E9000B10883E0A816B10488F5CE0144960E94FB
:100EA000054F882E912CA12CB12CCE0145960E9485
:100EB000054F482F50E060E070E08FEF88169104F6
:100EC000A104B104A9F44F3F51056105710581F4F6
:100ED0008FEF481651046104710481F48FEFC81636
:100EE000D104E104F10451F46FEF7FEFCB012BC08B
:100EF00040385105610571056CF0F6CF80E8C816E1
:100F0000D104E104F10484F740E050E0BA01812CFF
:100F1000912C5401FE2CED2CDC2CCC24C40CD51CC3
:100F2000E61CF71C540199248824C80CD91CEA1C1F
:100F3000FB1C742F662755274427CB01BA016C0D83
:100F40007D1D8E1D9F1DDF91CF91FF90EF90DF9053
:100F5000CF90BF90AF909F908F907F906F905F9059
:100F60004F9008950E944A1BFC01148680E090E097
:100F700008958FE994E00E94CB3B87E193E00E94C3
:100F8000CB3B0E944A1B0E94541A80E090E00895D7
:100F900080918B0B81113FC081E080938B0B0E946D
:100FA000C819FC01E159FF4F2081222369F0709795
:100FB00040815181628173814F5F5F4F6F4F7F4FDF
:100FC0004083518362837383FC01E751FF4F20818B
:100FD000222369F0709740815181628173814F5F54
:100FE0005F4F6F4F7F4F4083518362837383FC0158
:100FF000ED59FE4F2081222361F07097808191810D
:10100000A281B3810196A11DB11D80839183A2832A
:10101000B38310928B0B08950C94D7480C94D74847
:101020000C94D7480C94D7480C94D7480C94D748C4
:101030000C94D7480C94D7480C94D7480C94D748B4
:101040000C94D7480C94D7480C94D7480C94D748A4
:10105000CF93DF93EB0120E030E040E85FE36A816B
:101060007B818C819D810E94E94D811111C084EAB0
:1010700094E00E94CB3B0E94C819FC01E25BFF4F49
:10108000108211821282138282589E4F0E94123D5A
:1010900020E030E040E85FE36E817F8188859985BC
:1010A0000E94E94D811111C084EB94E00E94CB3B7A
:1010B0000E94C819FC01E853FF4F1082118212826E
:1010C000138286569E4F0E94123D20E030E040E899
:1010D0005FE36A857B858C859D850E94E94D811142
:1010E00011C084EC94E00E94CB3B0E94C819FC0123
:1010F000EE5BFE4F10821182128213828A549E4F41
:101100000E94123D0E944A1B0E94541A80E090E007
:10111000DF91CF9108958F929F92AF92BF92CF921D
:10112000DF92EF92FF920F931F930E94C81921E064
:101130002F931F921F921F921F92812C912CA12CF2
:10114000B12CC12CD12C760197018601B701A601E3
:1011500069D40F900F900F900F900F9080E090E067
:101160001F910F91FF90EF90DF90CF90BF90AF90C5
:101170009F908F9008950F931F93CF93DF938B01D0
:10118000EA01AB01415051094433510508F0D4C084
:101190002230310508F0D0C048E3429FF001439F60
:1011A000F00D1124E60FF71FE80FF91F81E080838F
:1011B000232B11F46C2F07C061E0802F0E94FA22CC
:1011C000209739F460E0802F0E94062280E090E0B2
:1011D000B5C0CF3FD10509F4ADC0F801E953FB4FCD
:1011E000E4918E2F90E0FC013197E231F10508F097
:1011F0009DC08827EE5AFE4F8F4F0C947E5084B5C9
:10120000806884BDC7BDE2CF84B5806284BDC8BD9F
:10121000DDCF80918000806880938000D09389002A
:10122000C0938800D3CF809180008062809380003B
:10123000D0938B00C0938A00C9CF809180008860D2
:1012400080938000D0938D00C0938C00BFCF80919D
:10125000B00080688093B000C093B300B7CF809196
:10126000B00080628093B000C093B400AFCF809193
:101270009000806880939000D0939900C09398006C
:10128000A5CF80919000806280939000D0939B00C6
:10129000C0939A009BCF80919000886080939000CB
:1012A000D0939D00C0939C0091CF8091A000806856
:1012B0008093A0008091A0008F7B8093A000D093AA
:1012C000A900C093A80082CF8091A0008062809383
:1012D000A000D093AB00C093AA0078CF8091A0006B
:1012E00088608093A000D093AD00C093AC006ECF17
:1012F00080912001806880932001D0932901C093C0
:10130000280164CF80912001806280932001D093D6
:101310002B01C0932A015ACF8091200188608093CD
:101320002001D0932D01C0932C0150CFC038D1059E
:101330000CF448CF61E047CF81E090E0DF91CF919E
:101340001F910F9108958F929F92AF92BF92CF926B
:10135000DF92EF92FF920F931F930E94C81960E0F3
:1013600070E00E94B536892BC9F40E94C8191F92FB
:101370001F9221E02F931F921F92812C912CA12C60
:10138000B12CC12CD12C760197018601B701A601A1
:1013900049D30F900F900F900F900F9080E090E046
:1013A0001F910F91FF90EF90DF90CF90BF90AF9083
:1013B0009F908F9008958F929F92AF92BF92CF92FD
:1013C000DF92EF92FF920F931F930E94C81961E082
:1013D00070E00E94B536892BC9F40E94C8191F928B
:1013E00021E02F931F921F921F92812C912CA12CF0
:1013F000B12CC12CD12C760197018601B701A60131
:1014000011D30F900F900F900F900F9080E090E00D
:101410001F910F91FF90EF90DF90CF90BF90AF9012
:101420009F908F900895CF92DF92EF92FF92CF938B
:10143000DF93EB010E941C36882359F1FE01EE0F69
:10144000FF1FEE0FFF1FE85AF84FC080D180E280E7
:10145000F38084ED94E00E94CB3B82EA94E00E940A
:10146000CB3B88ED94E00E94CB3BCE010E943E3CFA
:1014700082EA94E00E94CB3B8AED94E00E94CB3B51
:10148000C701B6010E94173C0E944A1B0E94541AD1
:1014900004C08CED94E00E94CB3B80E090E0DF91B3
:1014A000CF91FF90EF90DF90CF900895EF92FF9251
:1014B0000F931F93CF93DF9380918C0B90918D0BA3
:1014C000892B09F066C084E090E00E944248EC015C
:1014D00060E070E0BADC16161706FCF0CE014DDCB9
:1014E00098E5E92E97E0F92E00E010E0B801CE0172
:1014F0000E941C36882341F0F7012081318142810E
:101500005381B801CE0152DC0F5F1F4FF4E0EF0EA4
:10151000F11C0639110551F738C063E070E0CE01C7
:1015200094DC613071058105910569F588E5E82E47
:1015300087E0F82E00E010E0B801CE010E941C36D2
:101540008823C1F0B801CE0180DCF701608371838C
:10155000828393836F3F7F4F8F4F9F4F59F4B80122
:10156000CE0123D8F7012081318142815381B80116
:10157000CE011CDC0F5F1F4FF4E0EF0EF11C013EAB
:101580001105D1F602C0CE01F8DBD0938D0BC093CC
:101590008C0B80918C0B90918D0BDF91CF911F91D3
:1015A0000F91FF90EF900895EF92FF920F931F938A
:1015B000CF93DF9300D01F92CDB7DEB7FB0122A1FE
:1015C00033A144A155A1068D178D29833A834B83FE
:1015D0005C836CDF7C01FC018281938129813A81EB
:1015E0004B815C818F30F7E29F072CF40196F70165
:1015F0009383828303C0F70113821282B801C7016B
:1016000029833A834B835C830E941C3629813A816B
:101610004B815C81882391F0F801EE0FFF1FEE0FE4
:10162000FF1FE85AF84F2083318342835383B80168
:10163000C701BCDBB801C701F6DE04C08CED94E045
:101640000E94CB3B0E94FB1D0E94CB1D80E090E0DE
:101650000F900F900F900F90DF91CF911F910F91EE
:10166000FF90EF9008950F931F93CF93DF931EDFAA
:101670008C01C0E0D0E0BE01C8010E941C36882366
:1016800019F0BE01C801CFDE2196C13ED10599F700
:101690008EEF94E00E94CB3B0E944A1B0E94541A9A
:1016A00080E090E0DF91CF911F910F910895089510
:1016B00008950895EF92FF920F931F93CF93DF93B6
:1016C000162F072F7A014115510559F4862F0E94D4
:1016D000DE2131E020E0019709F030E0C32FD22F66
:1016E00026C04130510509F5262F663310F02AEC4B
:1016F000260F80917B00922F9870877F892B809393
:101700007B002770206420937C0080917A008064A5
:1017100080937A0080917A0086FDFCCFC09178009A
:1017200080917900D0E0D82B02C0C0E0D0E082E008
:10173000E816F10410F582E095E00E94CB3B82EAC6
:1017400094E00E94CB3B88ED94E00E94CB3B812F3C
:10175000902F0E943E3C82EA94E00E94CB3B8AEDAF
:1017600094E00E94CB3BCE010E943E3C0E944A1B6B
:101770000E94541A80E090E002C081E090E0DF9186
:10178000CF911F910F91FF90EF9008958091890B59
:1017900090918A0B892BA1F480E790E00E94424847
:1017A000FC01F9969C0123593F4FDF01D8971C9209
:1017B0001192E217F307C9F790938A0B8093890B74
:1017C0008091890B90918A0B089586E095E00E94A4
:1017D000CB3B0E944A1B0E948A1D0E944A1B0E940A
:1017E000661AD4DF40E050E068E070E063DFCEDFEF
:1017F00040E050E069E070E05DDFC8DF40E050E0CD
:101800006AE070E057DFC2DF40E050E06DE070E07A
:1018100051DF80E090E008956F927F928F929F92C7
:10182000AF92BF92CF92DF92EF92FF920F931F93EE
:10183000CF93DF93FB01E2A8F3A886A497A4A0A806
:10184000B1A8C6A0D7A062A073A0068D178D9EDF99
:10185000EC019701A301B8018EDCC501B4010E941F
:1018600041239701A601B801CE0185DC80E090E01C
:10187000DF91CF911F910F91FF90EF90DF90CF906C
:10188000BF90AF909F908F907F906F9008950F932F
:101890001F93CF93DF93FB0102A913A9C68DD78DA8
:1018A00075DFA801BE0106DF80E090E0DF91CF91F7
:1018B0001F910F9108951F93CF93DF931F92CDB780
:1018C000DEB7FB0162A9168D698360DF6981812F14
:1018D0000E94FA2280E090E00F90DF91CF911F915B
:1018E0000895EF92FF920F931F93CF93DF93FB0125
:1018F000E2A8F3A802A113A1C68DD78D47DF9701F7
:10190000A801BE0138DC80E090E0DF91CF911F910B
:101910000F91FF90EF900895089508950895089508
:101920000895CF93DF93FC01A489B589C08DD18D33
:101930002089318942895389A03187E2B80759F05B
:101940001A161B0644F40E94414F20E43CE940E093
:1019500050E00E941B4FDE010E94414FDF91CF916A
:101960000895FC0181E090E0938F828F11821082B4
:1019700015821482108A118A128A138A178A168A8B
:1019800080E197E2958B848B1286108614861586EB
:101990001686178608958EBD00000DB407FEFDCF94
:1019A0008EB50895CF92DF92EF92FF920F931F931F
:1019B000CF93DF93EC0160E086E10E9406228A8DDE
:1019C0009B8D24E0880F991F2A95E1F78F60E3DF54
:1019D00083E290E00197F1F704E010E0C12CD12CF4
:1019E0007601FE2CED2CDC2CCC2481E0D4DFC82A3F
:1019F00001501109B1F761E086E10E940622C88A10
:101A0000D98AEA8AFB8ADF91CF911F910F91FF90CB
:101A1000EF90DF90CF900895089508950895089568
:101A2000089508952F923F924F925F926F927F9206
:101A30008F929F92AF92BF92CF92DF92EF92FF92DE
:101A40000F931F93CF93DF93CDB7DEB7E0970FB619
:101A5000F894DEBF0FBECDBF1C012A013B010F83EE
:101A6000188729873A8728960EAD1FAD2897FC0165
:101A7000E55AFD4F60817181828193810E94EF4D13
:101A80009B01AC01C301B2010E944E4E0E94455021
:101A90006D877E878F87988BF101E15AFD4F6081BA
:101AA0007181828193810E94EF4D9B01AC016F8116
:101AB000788589859A850E944E4E0E9445506F8B8D
:101AC000788F898F9A8FF101ED59FD4F6081718177
:101AD000828193810E94EF4D9B01AC01C701B60149
:101AE0000E944E4E0E9445506B8F7C8F8D8F9E8F33
:101AF0000E9479236B8B7C8B8D8B9E8BF101E45242
:101B0000FE4F118210823296118210823E96A114ED
:101B1000B10461F0C501A0E0B0E040815181628173
:101B2000738184179507A607B70714F0A080B180CA
:101B3000F101E051FE4F8114910461F0C401A0E075
:101B4000B0E0408151816281738184179507A607B7
:101B5000B70714F080809180F101EC50FE4F011521
:101B6000110561F0C801A0E0B0E0408151816281BF
:101B7000738184179507A607B70714F000811181B8
:101B80009101205F3F4F3A8B298BC501A0E0B0E067
:101B9000F10180A791A7A2A7B3A72101FAE84F0EF0
:101BA000511CA12CB12CD20158968D929D92AD92D0
:101BB000BC925B973101BCEF6B1ABEEF7B0A20E051
:101BC00030E0F301008F118F228F338F0E944A1B68
:101BD0000E944A1B0E944A1B0E944A1B40914C07CC
:101BE00050914D0760914E0770914F074DA75EA72A
:101BF0006FA778AB0E944A1B8091500790915107C4
:101C0000A0915207B09153078F839887A987BA870D
:101C10000E944A1B8090540790905507A090560749
:101C2000B0905707F101E959FD4F108211821282DD
:101C3000138234961082118212821382349610829B
:101C4000118212821382349611821082329611828E
:101C5000108232961182108232964DA55EA56FA534
:101C600078A9408351836283738334968F819885EA
:101C7000A985BA8580839183A283B38334968082B9
:101C80009182A282B3822996EFAC29970D851E8599
:101C90002F85388989899A890E945A318823F9F0D9
:101CA00088E493E00E94CB3B81EB94E00E94CB3B25
:101CB000F101EE5AFF4F6081718182819381E75F6C
:101CC000FD4F20813181428153810E941B4FCA0107
:101CD000B9010E94173C0E944A1B0E94541A2A967E
:101CE000EFAC2A970F89188D298D3A8D4F81588531
:101CF00069857A85C2010E945A318823F9F084E40B
:101D000093E00E94CB3B81EC94E00E94CB3BF1013D
:101D1000E453FF4F6081718182819381ED56FE4FC4
:101D200020813181428153810E941B4FCA01B90138
:101D30000E94173C0E944A1B0E94541A2B96EFAC3B
:101D40002B970B8D1C8D2D8D3E8DB501A401C301EC
:101D50000E945A318823F9F080E493E00E94CB3B43
:101D600081ED94E00E94CB3BF101EA5BFE4F608184
:101D7000718182819381E35EFE4F208131814281B6
:101D800053810E941B4FCA01B9010E94173C0E9457
:101D90004A1B0E94541AD10151961C92F101E55739
:101DA000FF4F1082E658FF4F1082C1010E947D262E
:101DB000C1010E94812689899A890E949535C201B4
:101DC0000E949535C3010E94953581E090E0F101B4
:101DD000ED51FE4F918380837101BBE1EB1ABEEFA1
:101DE000FB0AF70191838083810109511E4FD801BD
:101DF0008D939C9341E050E069897A89C1010E94EA
:101E0000A21BF70140815181B201C1010E94A21BB6
:101E1000D8014D915C91B301C1010E94A21B11E058
:101E2000F101EE53FD4F108389899A890E94453153
:101E3000C2010E944531C3010E94453164E670E051
:101E400080E090E00E944123C10180529E4FFC013E
:101E50001083D101AF51BE4F1C93A1014E515E4F73
:101E6000FA0110832996FFAD2997F1110FC02A9628
:101E70002FAD2A97211105C02B963FAD2B97332309
:101E800039F1910121593F4FF90110822A96FFAD96
:101E90002A97F11105C0910127513F4FF901108296
:101EA0002B96FFAD2B97F11105C091012D593E4F97
:101EB000F901108229962FAD2997FC0120832A96DB
:101EC0003FAD2A973C932B96EFAD2B97DA01EC931D
:101ED00089899A890E940333C2010E940333C30196
:101EE0000E94033389899A890E945932C2010E9453
:101EF0005932C3010E9459320E944A1BDC011C96D0
:101F00008C918D8718861F82F101E052FE4FF88F69
:101F1000EF8B91012F513E4F3C8F2B8FA1014E51E2
:101F20005E4F58A34F8FC1018D519E4F9EA38DA32D
:101F3000D101AB51BE4FB8A7AFA3E655F140FAA30C
:101F4000E9A32D5D31093CA32BA3FE96FAA7E9A7CF
:101F5000225C3F4F3CA72BA7AF89B88D8C91811194
:101F60000BC0EB8DFC8D8081811106C0AF8DB8A1B7
:101F70008C91882309F459C3BD85B11156C3C101A1
:101F80000E945B264DA15EA169897A89C1010E94E8
:101F9000F21B4FA158A5B201C1010E94F21BA10181
:101FA00049515E4FB301C1010E94F21B89899A8990
:101FB0000E94C332C2010E94C332C3010E94C332D5
:101FC000F101EE58FF4F8081882341F189899A8978
:101FD0000E940333F101ED55FD4F80818823D1F03C
:101FE000610139E6C31A3DEFD30A71014EE4E41AE8
:101FF0004DEFF40A81010B571D4F910127583D4FBA
:10200000A10149595D4FB10162587E4F89899A8972
:102010000E949F25F101EE58FF4F1082F101E4511B
:10202000FF4F8081882331F1C2010E940333F10107
:10203000EC55FD4F80818823C9F0610155E6C51A32
:102040005DEFD50A71018CE4E81A8DEFF80A810181
:1020500007571D4F910123583D4FA10145595D4F31
:10206000B10166567E4FC2010E949F25F101E451E5
:10207000FF4F1082F101EA59FE4F8081882331F130
:10208000C3010E940333F101EB55FD4F808188238A
:10209000C9F0610191E6C91A9DEFD90A7101AAE45C
:1020A000EA1AADEFFA0A810103571D4F91012F572C
:1020B0003D4FA10141595D4FB1016A547E4FC301AB
:1020C0000E949F25F101EA59FE4F108281010159BA
:1020D0001F4FF80180818823E9F1EE5DFD4F60819B
:1020E0007181072E000C880B990B0E94EF4D9B010C
:1020F000AC01F101E959FD4F6081718182819381C9
:102100000E947650181634F5D8011C9266E274E0ED
:1021100081010E521E4FC8010E9428216BE475E018
:10212000C8010E9428216EE973E0C8010E9428219D
:102130002996BFAD2997BB2309F471C3C101825809
:102140009E4F0E94123DF101E25BFF4F108211820F
:1021500012821382810107511F4FD8018C9188236D
:1021600009F43EC0F101ED56FD4F60817181072EEB
:10217000000C880B990B0E94EF4D9B01AC01F10103
:10218000E559FD4F60817181828193810E94765073
:10219000181634F5D8011C9266E274E081010E52E3
:1021A0001E4FC8010E94282163E775E0C8010E9404
:1021B00028216EE973E0C8010E9428212A96BFAD4C
:1021C0002A97BB2309F430C3C10186569E4F0E9453
:1021D000123DE9A1FAA1FE961082118212821382A9
:1021E00081010D591E4FF80180818823E9F1EE5CD1
:1021F000FE4F60817181072E000C880B990B0E94A5
:10220000EF4D9B01AC01F101E159FD4F60817181FE
:10221000828193810E947650181634F5D8011C9261
:1022200066E274E081010E521E4FC8010E9428210F
:102230006BE975E0C8010E9428216EE973E0C801CE
:102240000E9428212B96BFAD2B97BB2309F4F1C226
:10225000C1018A549E4F0E94123DEBA1FCA1FE9643
:10226000108211821282138260E089899A890E9409
:10227000D231882361F0F101E25BFF4F10821182BD
:1022800012821382C10182589E4F0E94123D60E06B
:10229000C2010E94D231882361F0A9A5BAA51D927E
:1022A0001D921D921C921397C10186569E4F0E944B
:1022B000123D60E0C3010E94D231882359F0EBA5A2
:1022C000FCA51082118212821382C1018A549E4F92
:1022D0000E94123DF101E159FF4F8081AF89B88D15
:1022E0008C93E658FF4F8081EB8DFC8D8083F1014C
:1022F000ED59FE4F8081AF8DB8A18C93E551F1402F
:102300004081518162817381E9A1FAA1FE968080AA
:102310009180A280B380EBA1FCA1FE96C080D18009
:10232000E280F3804DA75EA76FA778AB0E944A1B9F
:102330004DA55EA56FA578A940934C0750934D0716
:1023400060934E0770934F070E944A1B809250077C
:1023500090925107A0925207B09253070E944A1BD5
:10236000C0925407D0925507E0925607F092570753
:10237000C1010E947D26EF89F88D8081882309F4B0
:102380004AC00E9479232B893C894D895E89621756
:1023900073078407950760F40E9479232B893C8991
:1023A0004D895E896217730784079507A0F51EC0E3
:1023B0000E9479236B017C012B893C894D895E89C0
:1023C000C21AD30AE40AF50AF101E15BFD4F20814C
:1023D000318142815381A8EEB3E00E94374F6C15E2
:1023E0007D058E059F0508F429C2D6CF0E9479236A
:1023F0006B017C01F101E15BFD4F20813181428164
:102400005381A8EEB3E00E94374F6C157D058E0511
:102410009F0508F413C2AB8DBC8D8C91882309F401
:102420004AC00E9479232B893C894D895E896217B5
:1024300073078407950760F40E9479232B893C89F0
:102440004D895E896217730784079507A0F51EC042
:102450000E9479236B017C012B893C894D895E891F
:10246000C21AD30AE40AF50AF101ED5AFD4F2081A0
:10247000318142815381A8EEB3E00E94374F6C1541
:102480007D058E059F0508F4F0C1D6CF0E94792303
:102490006B017C01F101ED5AFD4F208131814281B8
:1024A0005381A8EEB3E00E94374F6C157D058E0571
:1024B0009F0508F4DAC1AF8DB8A18C91882309F487
:1024C0004AC00E9479232B893C894D895E89621715
:1024D00073078407950760F40E9479232B893C8950
:1024E0004D895E896217730784079507A0F51EC0A2
:1024F0000E9479236B017C012B893C894D895E897F
:10250000C21AD30AE40AF50AF101E95AFD4F208103
:10251000318142815381A8EEB3E00E94374F6C15A0
:102520007D058E059F0508F4B7C1D6CF0E9479239B
:102530006B017C01F101E95AFD4F2081318142811B
:102540005381A8EEB3E00E94374F6C157D058E05D0
:102550009F0508F4A1C18BEA9BE00E94871E181614
:10256000190684F58BEA9BE00E94651E8F7D8534F9
:10257000910541F56DE075E0C1018E529E4F0E94BC
:10258000282184E693E00E94CB3B0E944A1B8CD713
:10259000F101E159FF4F1082E658FF4F1082E658D3
:1025A000FF4F1082AF89B88D1C92EB8DFC8D10828D
:1025B000AF8DB8A11C92B1E0BD87E1E0F0E0F887F3
:1025C000EF8304C02F813885232B81F062E275E010
:1025D000C1018E529E4F0E942821AF89B88D1C9256
:1025E000EB8DFC8D1082AF8DB8A11C92C1010E94B1
:1025F000813BF101E252FE4F8081918101969183EE
:1026000080838D3291400CF4A7CCD101AA52BE4FE9
:102610008D919C911197892B09F09ECC14968D91E8
:102620009C91892B09F44FC197CC81010A521E4F0E
:10263000F80180819181892B21F0C1010E94813BA9
:10264000F7CF82E395E00E94CB3B2996FFAD299717
:10265000FF2301F12F813885232BE1F43D853111D2
:102660003EC080E393E00E94CB3B0E944A1B1CD7F4
:102670002A964FAD2A97442369F18CE293E00E9499
:10268000CB3B0E944A1B10D72B965FAD2B97511165
:102690001AC025C02A968FAD2A97882341F0AF81B2
:1026A000B885AB2B21F4BD85B11119C0E6CF2B96AF
:1026B000EFAD2B97EE2399F02F813885232B79F4FA
:1026C0003D8531110CC088E293E00E94CB3BE2D7FC
:1026D000EBD605C02B969FAD2B979111F4CF8101BE
:1026E0000D511E4F85E090E0D8018D939C936101C0
:1026F000BBE1CB1ABEEFDB0AF60191838083710147
:10270000F9E1EF1AFEEFFF0AD7018D939C9345E0A4
:1027100050E069897A89C1010E94A21BF6014081BB
:102720005181B201C1010E94A21BD7014D915C9160
:10273000B301C1010E94A21BC1010E948526F101C3
:10274000E25BFF4F4081518162817381E658FF4F08
:1027500080809180A280B380E658FF4F8081918174
:10276000A281B3818B8B9C8BAD8BBE8B4DA75EA75B
:102770006FA778AB8FD74DA55EA56FA578A94093BD
:102780004C0750934D0760934E0770934F0782D7C5
:102790008092500790925107A0925207B09253072F
:1027A00079D72B893C894D895E89209354073093D2
:1027B00055074093560750935707C1010E947D2645
:1027C000C1010E94812666D7C2D6C1010E942A1C7F
:1027D000D8011D921C92F60111821082D7011D9220
:1027E0001C9240E050E069897A89C101ABD7F601BB
:1027F00040815181B201C101A5D7D7014D915C91B2
:10280000B301C1019FD7C1010E948526BD85BB23AD
:1028100009F424C23FD721E0FC0124871FC2E1E074
:10282000F0E0F887EF8396CCE1E0F0E0F887EF8303
:10283000D7CCE1E0F0E0F887EF8316CD6CE373E0EE
:1028400081010E521E4FC8010E9428216EE973E0DB
:10285000C8010E94282163EC75E0C8010E9428216C
:1028600022E030E038872F83D6CD68E373E0810122
:102870000E521E4FC8010E9428216EE973E0C80164
:102880000E94282168ED75E0C8010E94282142E0DD
:1028900050E058874F830FCE64E373E081010E52FE
:1028A0001E4FC8010E9428216EE973E0C8010E94F2
:1028B00028216DEE75E0C8010E94282182E090E099
:1028C00098878F8348CE11821082F101E452FE4F27
:1028D00080819181009749F460E673E081010E5296
:1028E0001E4FC8010E94282196C1019709F0A2C17C
:1028F000D1D68C01FC0180819181A281B38118160F
:1029000019061A061B0644F081E090E0A0E0B0E052
:1029100080839183A283B383F80184819581A6810A
:10292000B781181619061A061B0644F081E090E0DC
:10293000A0E0B0E084839583A683B783F801808507
:102940009185A285B385181619061A061B0644F050
:1029500081E090E0A0E0B0E080879187A287B38714
:1029600060EA73E0CE0101960E946B216EE275E091
:10297000CE0101960E94282161EB74E0CE01019600
:102980000E94282160914C0770914D0780914E075D
:1029900090914F070E94EF4D6B017C01D8016D9122
:1029A0007D918D919C910E94EF4D9B01AC01C701DF
:1029B000B6010E94DD4FAB01BC01CE0101960E9421
:1029C000982061EC74E0CE0101960E94282160916C
:1029D00050077091510780915207909153070E94C0
:1029E000EF4D6B017C01F8016481758186819781CF
:1029F0000E94EF4D9B01AC01C701B6010E94DD4F63
:102A0000AB01BC01CE0101960E94982061ED74E0FB
:102A1000CE0101960E9428216091540770915507BC
:102A200080915607909157070E94EF4D6B017C01F2
:102A3000D80118966D917D918D919C911B970E9464
:102A4000EF4D9B01AC01C701B6010E94DD4FAB0108
:102A5000BC01CE0101960E949820BE016F5F7F4F9E
:102A600081010E521E4FC8010E943621CE010196EF
:102A70000E9466210FD6BC01CE010196F9D4BE0199
:102A80006F5F7F4FC8010E943621CE0101960E94E0
:102A9000662164E273E0C8010E94282161EB74E0C2
:102AA000C8010E942821F101E258FE4FFC87EB8704
:102AB000CF010E94910C0E94EF4D6B017C01F1014E
:102AC000E55AFD4F60817181828193810E94EF4DB3
:102AD0009B01AC01C701B6010E94DD4FAB01BC01F7
:102AE000C8010E94C82061EC74E0C8010E9428213E
:102AF0006101F6E6CF1AFEEFDF0AC6010E94910CD3
:102B00000E94EF4D4B015C01F101E15AFD4F6081E4
:102B10007181828193810E94EF4D9B01AC01C501BF
:102B2000B4010E94DD4FAB01BC01C8010E94C82066
:102B300061ED74E0C8010E94282171012AE4E21AC3
:102B40002EEFF20AC7010E94910C0E94EF4D4B013B
:102B50005C01F101ED59FD4F6081718182819381AA
:102B60000E94EF4D9B01AC01C501B4010E94DD4FF5
:102B7000AB01BC01C8010E94C8208CD5BC01CE01AC
:102B8000019676D4BE016F5F7F4FC8010E94362147
:102B9000CE0101960E94662160E273E0C8010E94A6
:102BA000282161EB74E0C8010E942821EB85FC8597
:102BB000A08DB18D20893189428953890E94414F6E
:102BC000AB01BC01C8010E94F82061EC74E0C801AF
:102BD0000E942821F601A08DB18D2089318942897A
:102BE00053890E94414FAB01BC01C8010E94F820EB
:102BF00061ED74E0C8010E942821F701A08DB18D1C
:102C000020893189428953890E94414FAB01BC011F
:102C1000C8010E94F8203ED5BC01CE01019628D4FF
:102C2000BE016F5F7F4FC8010E943621CE01019621
:102C30000E946621F101E452FE4F8081918101964C
:102C4000823091051CF49183808302C0118210822E
:102C5000F101E652FE4F118210827EC980E495E0B8
:102C60000E94CB3B8F8198850E943E3C8EE993E089
:102C70000E94CB3B0FD52F81388530934707209397
:102C80004607C901E0960FB6F894DEBF0FBECDBF70
:102C9000DF91CF911F910F91FF90EF90DF90CF9038
:102CA000BF90AF909F908F907F906F905F904F906C
:102CB0003F902F900895662319F08FEA93E002C0A9
:102CC00088EA93E00C94CB3B0C94D7480C94D748FB
:102CD000CF92DF92EF92FF920F931F93CF93DF93E8
:102CE000EC018AE190E09E8B8D8B8BE190E0988FD8
:102CF0008F8B89E190E09A8F898F8FE090E09C8F95
:102D00008B8F8EE190E09E8F8D8F8EE090E098A368
:102D10008F8F85E490E09AA389A384E490E09CA33C
:102D20008BA3FE01E657FF4F80E290E096838583F8
:102D300081E290E0908787838FE190E0928781879E
:102D40001486138616861586108A178683E490E00B
:102D5000928B818B82E490E0948B838BE658FF4FBB
:102D600083E290E09683858384E290E09087878376
:102D700082E290E0928781871486138616861586F4
:102D8000108A178681E490E0928B818B80E490E03A
:102D9000948B838BE152FF4F118210823296118205
:102DA0001082329611821082CE010E948D28CE01AF
:102DB0000E94B226CE0182589E4F41E050E0FC01B5
:102DC000538F428FDE01A656BE4F24E030E05B9663
:102DD0003C932E935A976E01FAE4CF1AFEEFDF0A66
:102DE00028E030E0F601338F228F20E130E0FC0153
:102DF0003183208321E130E0358324832FEF3FEFBF
:102E00003383228337832683628560876385618766
:102E100067E170E011967C936E9368E170E015961F
:102E20007C936E93149713963C932E931297179658
:102E30003C932E9316971A966C911A9718966C934A
:102E400018971B966C911B9719966C9319976DE1C7
:102E500070E0F601718360836CE170E075836483D8
:102E60003383228337832683628560876385618706
:102E7000BE0168547D4FFB01608171818E01045554
:102E80001D4FF801008111817E01FAE5EF1AFDEF77
:102E9000FF0AF701E080F180FC01F78AE68A158BD2
:102EA000048B6130710519F4318F208F03C0FC0150
:102EB000518F408FCE0186549D4FFC0180819181BE
:102EC0009E0122553D4FF90120813181AE014855C7
:102ED0005D4FFA014081518157965C934E9356970E
:102EE00055963C932E935497019719F48FEF9FEFCB
:102EF00002C081E090E059969C938E935897DE0132
:102F0000A454BD4F8D919C9111971C972D913C918C
:102F1000C655DD4F48815981F601578B468B358B5D
:102F2000248B019719F48FEF9FEF03C081E090E0AD
:102F3000F601918F808FDF91CF911F910F91FF90BC
:102F4000EF90DF90CF9008952F923F924F925F9233
:102F50006F927F928F929F92AF92BF92CF92DF92A9
:102F6000EF92FF920F931F93CF93DF93CDB7DEB70E
:102F7000CA57D1090FB6F894DEBF0FBECDBF8C0182
:102F8000FC01108211821282138214821582168231
:102F90001782108611861286138614861586168669
:102FA00017862C01F0E14F0E511CC2010E94B7356B
:102FB00068018AE8C80ED11CC6010E94B7357801A5
:102FC000ECEFEE1AEEEFFE0AC7010E94B7353801AA
:102FD000F2E86F1AFEEF7F0AC3010E94B10C4801AC
:102FE00086E6881A8EEF980AC4010E94B10C580137
:102FF000EAE4AE1AEEEFBE0AC5010E94B10C60EA27
:1030000073E0C8018E529E4F0E946B21F801E85276
:10301000FE4F1182108232961182108232961182F6
:10302000108232961182108232961082319610826E
:10303000319610823196118210823296118210825E
:103040003296118210823296108231961082319619
:10305000108231961082118212821382349610826D
:10306000118212821382349610821182128213828C
:103070003496108211821282138234961082118249
:103080001282138234961082118212821382349635
:10309000108211821282138234961082118212825F
:1030A0001382349610821182128213823496108217
:1030B000118212821382349610821182128213823C
:1030C00034961082118212821382349610821182F9
:1030D00012821382349610821182128213823496E5
:1030E00010821182128213823496108231961082DD
:1030F0003196108231961082118212821382349698
:1031000010821182128213823496108211821282EE
:103110001382349610823196108231961082319645
:10312000108231961082319610823196108231963B
:10313000108231961082319610823196108231962B
:10314000108231961082319610823196108231961B
:10315000108231961082319610823196108231960B
:1031600010823196108231961082319610823196FB
:10317000108231961082118212821382349610824C
:10318000118212821382349610821182128213826B
:10319000D801A55ABD4F8CE0ECE4F3E001900D920C
:1031A0008A95E1F7F801E959FD4F108211821282E8
:1031B0001382349610821182128213823496108206
:1031C00011821282138234961182108232961182F9
:1031D00010823296118210823296108211821282EF
:1031E00013823496108211821282138234961082D6
:1031F00011821282138234961082118212821382FB
:1032000034961082118212821382349610821182B7
:1032100012821382349611821082329611821082A9
:10322000329611821082329610821182128213829B
:103230003496108211821282138234961082118287
:103240001282138234961082319610823196108247
:10325000319611821082329611821082329611823A
:10326000108232961182108232961182108232962A
:10327000118210823296118210823296118210824F
:103280003296118210823296118210823296118209
:1032900010823296118210823296118210823296FA
:1032A000118210821801FEE32F1AFDEF3F0AF1018F
:1032B0001082CE0101960E94B7358AE7FE01319651
:1032C000D20101900D928A95E1F7CE0101960E94FC
:1032D000B7358AE7FE013196D60101900D928A95A5
:1032E000E1F7CE0101960E94B7358AE7FE013196DB
:1032F000D70101900D928A95E1F788E5F801808B5E
:1033000089E5F60180838AE5F7018083CE01019685
:103310000E94B10C8CE1FE013196D30101900D9217
:103320008A95E1F7CE0101960E94B10C8CE1FE0175
:103330003196D40101900D928A95E1F7CE01019664
:103340000E94B10C8CE1FE013196D50101900D92E5
:103350008A95E1F7C801BCDCF1011082C658DF4F45
:103360000FB6F894DEBF0FBECDBFDF91CF911F9196
:103370000F91FF90EF90DF90CF90BF90AF909F9014
:103380008F907F906F905F904F903F902F90089517
:10339000CF93DF9380919A0B90919B0B892B51F4E3
:1033A00083EC92E00E944248EC01CEDDD0939B0B6F
:1033B000C0939A0B80919A0B90919B0BDF91CF91C8
:1033C00008954F925F926F927F928F929F92AF92E9
:1033D000BF92CF92DF92EF92FF920F931F93CF9302
:1033E000DF9300D01F92CDB7DEB7FB0116890789A6
:1033F00082889388A684B784C284D384E484F584C5
:1034000046805780608471844281538164817581D4
:1034100049835A836B837C83BBDF1F921F921F9269
:103420000F931F939301820149815A816B817C81A3
:103430000E94120D0F900F900F900F900F9080E050
:1034400090E00F900F900F900F90DF91CF911F9110
:103450000F91FF90EF90DF90CF90BF90AF909F9033
:103460008F907F906F905F904F900895089508958A
:10347000CF93DF93EC0160EA73E02DD762E076E052
:10348000CE01E6D6409148075091490760914A071E
:1034900070914B07CE01ACD66EE973E0CE01D8D661
:1034A000CE01DF91CF91089582E096E00E94CB3B60
:1034B000609148077091490780914A0790914B07A6
:1034C0000E94173C8EE993E00C94CB3B0F931F9323
:1034D000CF93DF93EC0185E096E00E94CB3B89E03F
:1034E00096E00E94CB3B04E91BE0F8016081CE012D
:1034F000E2DB8DE096E00E94CB3BF8016181CE01DA
:10350000DADB81E196E00E94CB3BF8016281CE01DB
:10351000D2DB85E196E00E94CB3BF8016381CE01CE
:10352000CADB89E196E00E94CB3BF8016481CE01C1
:10353000C2DB8DE196E00E94CB3BF8016581CE01B4
:10354000BADBCE01DF91CF911F910F91ADCFCF921A
:10355000DF92EF92FF92CF93DF93EC018881998104
:10356000AA81BB81181619061A061B0644F081E0D1
:1035700090E0A0E0B0E088839983AA83BB838C812C
:103580009D81AE81BF81181619061A061B0644F0EC
:1035900081E090E0A0E0B0E08C839D83AE83BF83A8
:1035A00088859985AA85BB85181619061A061B06F3
:1035B00044F081E090E0A0E0B0E088879987AA8796
:1035C000BB878EE295E00E94CB3B81EB94E00E94AA
:1035D000CB3B60914C0770914D0780914E079091C5
:1035E0004F070E94EF4D6B017C01688179818A81D0
:1035F0009B810E94EF4D9B01AC01C701B6010E9467
:10360000DD4F42E00E94433C81EC94E00E94CB3BC2
:103610006091500770915107809152079091530724
:103620000E94EF4D6B017C016C817D818E819F81B9
:103630000E94EF4D9B01AC01C701B6010E94DD4F16
:1036400042E00E94433C81ED94E00E94CB3B6091BC
:1036500054077091550780915607909157070E9423
:10366000EF4D6B017C01688579858A859B850E9479
:10367000EF4D9B01AC01C701B6010E94DD4F42E056
:103680000E94433CCE01DF91CF91FF90EF90DF90FD
:10369000CF900ACF8091920B9091930B892B91F54B
:1036A0008DE090E00E944248FC01148610924C0785
:1036B00010924D0710924E0710924F07109250072C
:1036C000109251071092520710925307109254070C
:1036D0001092550710925607109257071092910BAF
:1036E0001092900B109248071092490710924A07C7
:1036F00010924B0710924707109246079093930B36
:103700008093920B8091920B9091930B08950F935D
:103710001F93CF93DF938B01EA018CE593E00E9426
:10372000CB3B82EA94E00E94CB3BF80180810E946F
:103730000C3CCE010E943E3CADDFDF91CF911F914A
:103740000F91B2CECF92DF92EF92FF920F931F9321
:10375000CF93DF93CDB7DEB728970FB6F894DEBFCF
:103760000FBECDBF8B016A018E529E4F7C0168E572
:1037700073E06ED562EA74E0C7016AD5F801808112
:1037800089831A8241E050E08E010F5F1F4FB8011C
:10379000C701A1D44AE0B801C6010E949C49F801C2
:1037A00001900020E9F73197AF01401B510BB801A0
:1037B000C70191D46FDFBC01C8015ADEB801C7014F
:1037C00055D5C80183D528960FB6F894DEBF0FBE35
:1037D000CDBFDF91CF911F910F91FF90EF90DF90C0
:1037E000CF900895FC01DB01AD59BF4F8C91882328
:1037F00019F022E030E002C020E030E0DB01AB59FC
:10380000BF4F8C91882311F023E030E0DB01AC59ED
:10381000BF4F8C91882311F024E030E0DB01AA59DE
:10382000BF4F8C91882311F026E030E0DA018D91B2
:103830009C918217930721F091E0121613060CF069
:1038400090E0DA012D933C93992319F0A901CF015F
:1038500079CF08958F929F92AF92BF92CF92DF92CD
:10386000EF92FF920F931F93CF93DF93EC0184E2CB
:1038700093E00E94CB3B81EB94E00E94CB3B6E0136
:1038800082E8C81A8EEFD80AC6010E94910C0E94E5
:10389000EF4D4B015C01FE01E55AFD4F60817181E6
:1038A000828193810E94EF4D9B01AC01C501B4015F
:1038B0000E94DD4F42E00E94433C81EC94E00E9474
:1038C000CB3B7E01E6E6EE1AEEEFFE0AC7010E9450
:1038D000910C0E94EF4D4B015C01FE01E15AFD4F3E
:1038E00060817181828193810E94EF4D9B01AC01C7
:1038F000C501B4010E94DD4F42E00E94433C81EDCE
:1039000094E00E94CB3B8E010A541E4FC8010E94D6
:10391000910C0E94EF4D4B015C01CD59DD4F688148
:1039200079818A819B810E94EF4D9B01AC01C50189
:10393000B4010E94DD4F42E00E94433CABDEB4DDA7
:1039400080E293E00E94CB3B81EB94E00E94CB3B72
:10395000F601A08DB18D20893189428953890E9459
:10396000414F0E94173C81EC94E00E94CB3BF70151
:10397000A08DB18D20893189428953890E94414FA0
:103980000E94173C81ED94E00E94CB3BF801A08D92
:10399000B18D20893189428953890E94414F0E940B
:1039A000173C78DEDF91CF911F910F91FF90EF9040
:1039B000DF90CF90BF90AF909F908F9075CD4F923A
:1039C0005F926F927F928F929F92AF92BF92CF92AF
:1039D000DF92EF92FF920F931F93CF93DF9300D06C
:1039E0001F92CDB7DEB70E94560A4090340850901F
:1039F000350860903608709037080E94560A80900B
:103A0000380890903908A0903A08B0903B0842DE00
:103A1000C0904C07D0904D07E0904E07F0904F07B4
:103A200039DEC701B6010E94EF4D6B017C01C30175
:103A3000B2010E94EF4D9B01AC01C701B6010E948B
:103A4000DD4F2B013C01609150077091510780912F
:103A50005207909153070E94EF4D6B017C01C50105
:103A6000B4010E94EF4D9B01AC01C701B6010E9459
:103A7000DD4FAB01BC0149835A836B837C8388DCB7
:103A80001F921F921F921F921F92812C912CA12C8A
:103A9000B12CC12CD12C760149815A816B817C815A
:103AA0008A019B01B301A2010E94120D71DC1F92D9
:103AB0001F921F921F921F9297018601B301A201CC
:103AC0000E94120D65DC1F921F921F921F921F927F
:103AD00097018601B701A6010E94120D0FB6F89456
:103AE000DEBF0FBECDBF80E090E00F900F900F9033
:103AF0000F90DF91CF911F910F91FF90EF90DF908A
:103B0000CF90BF90AF909F908F907F906F905F907D
:103B10004F900895CF93DF9385E450D4EC01BADD44
:103B200091E0CD2B09F490E09093940B84E446D47B
:103B3000EC01B0DD91E0CD2B09F490E09093950B72
:103B400083E43CD4EC01A6DD91E0CD2B09F490E0B8
:103B50009093960B82E432D4EC019CDD91E0CD2B66
:103B600009F490E09093970B81E428D4EC0192DD66
:103B700091E0CD2B09F490E09093980B80E41ED453
:103B8000EC0188DD91E0CD2B09F490E09093990B46
:103B9000DF91CF910895CF93DF93EC012AEC30E0D1
:103BA0004BEC50E069EC70E07BD72EEC30E04FEC52
:103BB00050E06DEC70E0CE010C9672D724ED30E051
:103BC00045ED50E063ED70E0CE01489669D728EDF1
:103BD00030E049ED50E067ED70E0CE01849660D7AB
:103BE0002EED30E04FED50E06DED70E0CE01C0966F
:103BF000DF91CF9155C7CF93DF9380918E0B90913A
:103C00008F0B892BE9F48CE390E00E944248EC0191
:103C1000FC01CC96118210823C96E817F907D1F787
:103C2000198218821D861C86198E188E1DA21CA250
:103C300019AA18AACE01AFDFD0938F0BC0938E0BB9
:103C400080918E0B90918F0BDF91CF910895CF9241
:103C5000DF92EF92FF920F931F93CF93DF936C014C
:103C60007A018B01C0E0D0E0CE15DF0589F0D801E4
:103C70006D918D01D601ED91FC910190F081E02DC7
:103C8000C6011995892B11F47E0102C02196ECCF53
:103C9000C701DF91CF911F910F91FF90EF90DF90BF
:103CA000CF900895089580E090E00895FC01538D31
:103CB000448D252F30E0842F90E0821B930B541706
:103CC00010F0CF96089501970895FC01918D828D93
:103CD000981761F0828DDF01A80FB11D5D968C9160
:103CE000928D9F5F9F73928F90E008958FEF9FEF6B
:103CF0000895FC01918D828D981731F0828DE80F27
:103D0000F11D858D90E008958FEF9FEF0895FC01E0
:103D1000918D228D892F90E0805C9F4F821B9109AD
:103D20008F73992708958BEA9BE0F1DF21E0892BBF
:103D300009F420E0822F0895FC01848DDF01A80F93
:103D4000B11DA35ABF4F2C91848D90E001968F73C3
:103D50009927848FA689B7892C93A089B1898C91E2
:103D600080648C93938D848D981306C00288F389A8
:103D7000E02D80818F7D80830895EF92FF920F93D5
:103D80001F93CF93DF93EC0181E0888F9B8D8C8D07
:103D9000981305C0E889F989808185FD23C0F62E36
:103DA0000B8D10E00F5F1F4F0F731127E02E8C8DCE
:103DB000E8120BC00FB607FCFACFE889F9898081B9
:103DC00085FFF5CFCE01B8DFF2CF8B8DFE01E80F76
:103DD000F11DE35AFF4FF0820B8FEA89FB89808146
:103DE000806207C0EE89FF896083E889F989808154
:103DF0008064808381E090E0DF91CF911F910F91EB
:103E0000FF90EF900895CF93DF93EC01888D882386
:103E1000C1F0EA89FB89808185FD05C0A889B9893F
:103E20008C9186FD0EC00FB607FCF5CF808185FF13
:103E3000F2CFA889B9898C9185FFEDCFCE017CDFC7
:103E4000E8CFDF91CF91089580E090E0892B19F0C1
:103E50006ADF811125C080E090E0892B41F080E08D
:103E600090E0892B21F00E94000081111CC080E0AD
:103E700090E0892B41F080E090E0892B21F00E94B6
:103E80000000811113C080E090E0892BA1F080E058
:103E900090E0892B81F00E94000081110AC00895F2
:103EA0000E940000D8CF0E940000E1CF0E940000D5
:103EB000EACF0C940000089590E0FC013197E231C4
:103EC000F10508F04EC08827EC59FE4F8F4F0C9437
:103ED0007E50809180008F7703C0809180008F7D1D
:103EE00080938000089580918000877FF9CF84B50A
:103EF0008F7702C084B58F7D84BD08958091B00016
:103F00008F7703C08091B0008F7D8093B0000895BB
:103F1000809190008F7707C0809190008F7D03C0C3
:103F200080919000877F8093900008958091A000F9
:103F30008F7707C08091A0008F7D03C08091A00083
:103F4000877F8093A0000895809120018F7707C01C
:103F5000809120018F7D03C080912001877F809315
:103F6000200108953FB7F8948091A50B9091A60B7E
:103F7000A091A70BB091A80B26B5A89B05C02F3F19
:103F800019F00196A11DB11D3FBFBA2FA92F982F7F
:103F90008827820F911DA11DB11DBC01CD0142E0FA
:103FA000660F771F881F991F4A95D1F708950E94C1
:103FB0006D510C94D7480C94D7480F931F93CF930F
:103FC000DF93EC0188819981009729F02A813B8158
:103FD0002617370788F48B016F5F7F4F0E9486504A
:103FE000009761F0998388831B830A832C813D812C
:103FF000232B11F4FC01108281E001C080E0DF91ED
:10400000CF911F910F9108958F929F92AF92BF927F
:10401000CF92DF92EF92FF920F931F93B9D962E094
:1040200070E00E94B536892BC9F4B2D921E02F93F4
:104030001F921F921F921F92812C912CA12CB12CA8
:10404000C12CD12C760197018601B701A6010E94EF
:10405000120D0F900F900F900F900F9080E090E056
:104060001F910F91FF90EF90DF90CF90BF90AF9096
:104070009F908F9008958F929F92AF92BF92CF9210
:10408000DF92EF92FF920F931F9382D91F9221E04C
:104090002F931F921F921F92812C912CA12CB12C37
:1040A000C12CD12C760197018601B701A6010E948F
:1040B000120D0F900F900F900F900F9080E090E0F6
:1040C0001F910F91FF90EF90DF90CF90BF90AF9036
:1040D0009F908F900895EF92FF920F931F93CF932D
:1040E000DF93FC01248135816115710511F480E0B5
:1040F00018C041155105A1F07B01EC018A01020FA6
:10410000131FB8015ADF882391F3288139818C81EC
:104110009D81B701820F931F0E9483511D830C83E1
:1041200081E0DF91CF911F910F91FF90EF90089563
:10413000EF92FF920F931F93CF93DF93CDB7DEB72C
:1041400064970FB6F894DEBF0FBECDBF7C01CB01E4
:10415000BA018E010F5F1F4F22E044E00E94234806
:10416000BC01FC0101900020E9F73197AF01481B29
:10417000590BC701B0DF64960FB6F894DEBF0FBECF
:10418000CDBFDF91CF911F910F91FF90EF900895D8
:10419000EF92FF920F931F93CF93DF93CDB7DEB7CC
:1041A00064970FB6F894DEBF0FBECDBF7C01CB0184
:1041B000BA018E010F5F1F4F22E044E00E942348A6
:1041C000BC01FC0101900020E9F73197AF01481BC9
:1041D000590BC70180DF64960FB6F894DEBF0FBE9F
:1041E000CDBFDF91CF911F910F91FF90EF90089578
:1041F000EF92FF920F931F93CF93DF93CDB7DEB76C
:104200002E970FB6F894DEBF0FBECDBF7C01CB0159
:10421000BA012AE08E010F5F1F4FA8010E94A64934
:10422000F80101900020E9F73197AF01401B510BD5
:10423000B801C70150DF2E960FB6F894DEBF0FBE4F
:10424000CDBFDF91CF911F910F91FF90EF90089517
:104250006115710549F0FB0101900020E9F73197E4
:10426000AF01461B570B37CF80E00895FB01448117
:104270005581608171812FCFEF92FF920F931F9331
:10428000CF93DF93EC017B018A01BA0196DE28818E
:10429000398181110DC02115310519F0C9010E9424
:1042A000D748198218821D821C821B821A8206C07E
:1042B0001D830C83B701C9010E948351CE01DF9198
:1042C000CF911F910F91FF90EF900895FC01808195
:1042D00091810C94D748FC011182108213821282C2
:1042E000158214826115710549F0FB0101900020CF
:1042F000E9F73197AF01461B570BBECF08951F92C8
:104300000F920FB60F9211240BB60F922F933F937B
:104310004F935F936F937F938F939F93AF93BF93CD
:10432000EF93FF938BEA9BE007DDFF91EF91BF9145
:10433000AF919F918F917F916F915F914F913F913D
:104340002F910F900BBE0F900FBE0F901F901895DE
:104350001F920F920FB60F9211240BB60F922F934C
:104360008F939F93EF93FF93E091BB0BF091BC0B66
:104370008081E091C10BF091C20B82FD12C090814F
:104380008091C40B8F5F8F732091C50B821751F002
:10439000E091C40BF0E0E555F44F958F8093C40B8A
:1043A00001C08081FF91EF919F918F912F910F908C
:1043B0000BBE0F900FBE0F901F901895CF93DF93F9
:1043C000282F30E0F901E953FB4F8491F901E55CB6
:1043D000FB4FD491F901EF57FB4FC491CC2389F0E7
:1043E00081116ADDEC2FF0E0EE0FFF1FE95DFA4F5F
:1043F000A591B491EC91ED2381E090E021F480E06F
:1044000002C080E090E0DF91CF9108951F93CF9399
:10441000DF93282F30E0F901E953FB4F8491F90134
:10442000E55CFB4FD491F901EF57FB4FC491CC23CE
:10443000C1F0162F811140DDEC2FF0E0EE0FFF1FD1
:10444000E35FFA4FA591B4918FB7F894111105C0AD
:104450009C91ED2FE095E92302C0EC91ED2BEC93BC
:104460008FBFDF91CF911F910895CF92DF92EF928E
:10447000FF920F931F93CF93DF936C018B017A010F
:10448000EC01C456D44F888187FF04C0FB01118220
:10449000108224C08CE08C9D90018D9D300D1124E4
:1044A0008881A901480F511D87FD5A958091E00C24
:1044B00090E04817590794F48881A901480F511DCD
:1044C00087FD5A95CA01FA01EE0FFF1F8E0F9F1F3D
:1044D000FC01E05BF34F808186FD19C088818F5F0E
:1044E00088838CE08C9D90018D9D300D11248881F6
:1044F000A901480F511D87FD5A958091E00C90E06D
:1045000048175907B4F488818C303CF112C0888177
:10451000280F311D87FD3A95F901EE0FFF1F2E0F71
:104520003F1FF901E05BF34F808160E08F736EDF26
:10453000D5CFF80180819181049680349C4918F48C
:1045400080E49CE904C0F801808191810496F70120
:10455000918380838FEF888344C0F801408151812B
:104560008881B901680F711D87FD7A95CB01FB0128
:10457000EE0FFF1F8E0F9F1FFC01E05BF34F818149
:104580009281840F951FF701918380838881A9010F
:10459000480F511D87FD5A95CA01FA01EE0FFF1F02
:1045A0008E0F9F1FFC01E05BF34F808186FF19C0D7
:1045B0008881280F311D87FD3A95F901EE0FFF1F05
:1045C0002E0F3F1FF901E05BF34F808161E08F7395
:1045D000DF91CF911F910F91FF90EF90DF90CF90DF
:1045E00015CFDF91CF911F910F91FF90EF90DF904A
:1045F000CF900895CF93DF9390E0FC01E55CFB4FF3
:104600002491FC01EF57FB4F8491882361F190E0E6
:10461000880F991FFC01EF5DFB4FC591D491FC0100
:10462000E35FFA4FA591B491611109C09FB7F89467
:104630008881209582238883EC912E230BC06230E1
:1046400061F49FB7F8943881822F80958323888303
:10465000EC912E2B2C939FBF06C08FB7F894E88166
:104660002E2B28838FBFDF91CF9108958230910543
:1046700038F0880F991F880F991F05970197F1F758
:1046800008958F929F92AF92BF92CF92DF92EF9256
:10469000FF926B017C0166DC4B015C01C114D1040B
:1046A000E104F104E9F05EDCDC01CB018819990931
:1046B000AA09BB09883E9340A105B10578F321E022
:1046C000C21AD108E108F10888EE880E83E0981E2E
:1046D000A11CB11CC114D104E104F10421F7DECF07
:1046E000FF90EF90DF90CF90BF90AF909F908F9012
:1046F00008952FB7F8946091A10B7091A20B80914F
:10470000A30B9091A40B2FBF08951F920F920FB689
:104710000F9211242F933F938F939F93AF93BF9347
:104720008091A10B9091A20BA091A30BB091A40B2F
:104730003091A00B23E0230F2D3720F40196A11D0B
:10474000B11D05C026E8230F0296A11DB11D2093BF
:10475000A00B8093A10B9093A20BA093A30BB093FB
:10476000A40B8091A50B9091A60BA091A70BB091E3
:10477000A80B0196A11DB11D8093A50B9093A60BCC
:10478000A093A70BB093A80BBF91AF919F918F916E
:104790003F912F910F900FBE0F901F901895CF92C1
:1047A000DF92EF92FF92CF93DF93EC01603282E0D1
:1047B00078070CF03DC077FD06C0653B71052CF015
:1047C00064EB70E002C060E070E0898128E830E0CE
:1047D0006901C81AD10887FDD394CC0CDD1CCC0C20
:1047E000DD1C0D2C000CEE08FF088A8128E532E064
:1047F000281B310987FD3395220F331F220F331FEA
:10480000C901330FAA0BBB0B9C01AD012C193D094B
:104810004E095F09DB010E94414F24EB30E040E08C
:1048200050E00E941B4FC20ED31EE41EF51EB601BF
:104830008881803380F5998148E850E0491B51090F
:1048400097FD5395440F551F440F551F6417750767
:1048500084F09A8128E532E0291B310997FD3395D0
:10486000220F331F220F331FAB01261737070CF41B
:10487000A90142505109440F551F2FB7F89490E0F9
:10488000FC01EE0FFF1F8E0F9F1FFC01E05BF34F3B
:10489000528341832FBFDF91CF91FF90EF90DF9044
:1048A000CF9008951F920F920FB60F9211240BB65E
:1048B0000F922F933F934F935F936F937F938F93B9
:1048C0009F93AF93BF93EF93FF9348E251E064E26D
:1048D00071E080E090E0C9DDFF91EF91BF91AF9171
:1048E0009F918F917F916F915F914F913F912F9108
:1048F0000F900BBE0F900FBE0F901F9018951F9238
:104900000F920FB60F9211240BB60F922F933F9375
:104910004F935F936F937F938F939F93AF93BF93C7
:10492000EF93FF9348EA50E064EA70E083E090E0A0
:104930009CDDFF91EF91BF91AF919F918F917F91FE
:104940006F915F914F913F912F910F900BBE0F9000
:104950000FBE0F901F9018951F920F920FB60F92D7
:1049600011240BB60F922F933F934F935F936F9346
:104970007F938F939F93AF93BF93EF93FF9348E9F8
:1049800050E064E970E082E090E06FDDFF91EF912C
:10499000BF91AF919F918F917F916F915F914F9157
:1049A0003F912F910F900BBE0F900FBE0F901F9055
:1049B00018951F920F920FB60F9211240BB60F92FB
:1049C0002F933F934F935F936F937F938F939F9317
:1049D000AF93BF93EF93FF9348E850E064E870E033
:1049E00081E090E042DDFF91EF91BF91AF919F9107
:1049F0008F917F916F915F914F913F912F910F9088
:104A00000BBE0F900FBE0F901F90189508950F9337
:104A10001F93CF93DF93FC01208131812115310554
:104A2000D1F1EC01822FCADC21E0892B09F420E0CE
:104A30002B876A85261729F01E821F821886198601
:104A40000BC08E819F81A885B9850196A11DB11DDE
:104A50008E839F83A887B9870E811F81288539851A
:104A60008A819B81AC81BD81081719072A073B0702
:104A700094F081E068278881C9DC0990D881C02D35
:104A80000E94C60B40E050E0BE01DF91CF911F9124
:104A90000F910C945A0BDF91CF911F910F910895B4
:104AA000CF92DF92EF92FF920F931F93CF93DF93FA
:104AB0007C016B018A01E9010E94560AF601EE0FA2
:104AC000FF1FEE0FFF1FE85AF84F80819181F70119
:104AD000918380830E94560A000F111F000F111F3F
:104AE000F801E85AF84F81E0408151816281738179
:104AF000413051056105710509F080E0F7018287B9
:104B00000E94560ACC0FDD1FCC0FDD1FC85AD84FAC
:104B100088819981AA81BB81F70182839383A483D1
:104B2000B5831682178210861186DF91CF911F916F
:104B30000F91FF90EF90DF90CF90089508952F92FE
:104B40003F924F925F926F927F928F929F92AF921D
:104B5000BF92CF92DF92EF92FF920F931F93CF936A
:104B6000DF9300D000D0CDB7DEB79E838D834B019D
:104B70005A013A8329831801FC82EB82FA014080B2
:104B800051806280738020E030E0A901C301B2014E
:104B90000E947650181674F4F6012081318142810A
:104BA0005381C301B2010E94784FF5016083718384
:104BB00082839383ED81FE81E05AFF4F8081F4016F
:104BC000008D118DC088D188E288F388F101408082
:104BD000518062807380D801A7019601882341F03B
:104BE0000E94414F641575058605970544F023C062
:104BF0000E94414F4616570668067906E4F4F5010F
:104C0000408051806280738020E030E04AEF56E4BB
:104C1000C301B2010E94E94D87FF0DC020E030E0E2
:104C200040E85FE3C301B2010E94794FF501608360
:104C3000718382839383D801A70196010E94414F1B
:104C4000F10160837183828393830D811E81025CF5
:104C50001F4FF80180819181A281B381E981FA819E
:104C600080839183A283B383EB81FC8180819181D6
:104C7000892B41F0C4010E94910CF801608371837B
:104C80008283938326960FB6F894DEBF0FBECDBF06
:104C9000DF91CF911F910F91FF90EF90DF90CF9018
:104CA000BF90AF909F908F907F906F905F904F904C
:104CB0003F902F900895CF93DF93EC0183B183B1A0
:104CC000E0E0F1E080818081CE0182589E4F0E9419
:104CD000D20C83B183B180B180B1CE0186569E4F94
:104CE0000E94D20C83B183B180B180B1CE018A54CD
:104CF0009E4FDF91CF910C94D20C0E944A1B0C94D2
:104D00008A1D0E944A1B0C94661ACF93DF93EC0114
:104D1000FC01EE53FD4F1082E858F10980818111AA
:104D200004C0CE0140960E943131FE01E55CFD4F8A
:104D30008081811105C0CE0186579F4F0E9431317D
:104D4000FE01E45CFD4F8081811105C0CE018C5FC6
:104D50009E4F0E94313164E670E080E090E0DF9188
:104D6000CF918FCC2F923F924F925F926F927F9212
:104D70008F929F92AF92BF92CF92DF92EF92FF926B
:104D80000F931F93CF93DF93EC010E94560AFE010D
:104D9000EF56FD4F809114099091150991838083FE
:104DA0000E94560AFE01ED56FD4F80911809909120
:104DB0001909918380830E94560AFE01EB56FD4F2C
:104DC00080911C0990911D09918380830E94560A4D
:104DD0008E0109561D4F60913C0970913D098091EB
:104DE0003E0990913F090E94EF4DF8016083718365
:104DF000828393830E94560A1E01F5E62F1AFDEF67
:104E00003F0A609140097091410980914209909157
:104E100043090E94EF4DF101608371838283938384
:104E20000E94560A20E030E048EC52E4F80160812C
:104E30007181828193810E94DD4F2B013C0120E032
:104E400030E048EC52E4F10160817181828193810C
:104E50000E94DD4F4B015C0160914409709145094E
:104E600080914609909147090E94EF4D20E030E083
:104E700048EC52E40E94DD4F6B017C012AE037EDE3
:104E800043E25CE3C301B2010E94765018168CF431
:104E900020E030E046EC52E4C301B2010E94E94D4B
:104EA00087FD0FC0412C512C46EC642E42E4742E39
:104EB00008C05AE0452E57ED552E53E2652E5CE3AF
:104EC000752EF80140825182628273822AE037EDAA
:104ED00043E25CE3C501B4010E94765018168CF4DD
:104EE00020E030E046EC52E4C501B4010E94E94DF7
:104EF00087FD0FC0812C912C26ECA22E22E4B22E2D
:104F000008C03AE0832E37ED932E33E2A32E3CE324
:104F1000B32EF10180829182A282B3822AE037ED22
:104F200043E25CE3C701B6010E94765018168CF488
:104F300020E030E046EC52E4C701B6010E94E94DA2
:104F400087FD0FC0C12CD12C86ECE82E82E4F82E10
:104F500008C09AE0C92E97EDD92E93E2E92E9CE382
:104F6000F92EFE01E156FD4FC082D182E282F3822A
:104F70000E94560A8091FC089091FD08FE01EA55B6
:104F8000FD4F918380830E94560A80910009909181
:104F90000109FE01E855FD4F918380830E94560A66
:104FA0008091040990910509FE01E655FD4F91831A
:104FB00080830E94560A8091240990912509FE0160
:104FC000E455FD4F918380830E94560A8091280901
:104FD00090912909FE01E255FD4F918380830E9443
:104FE000560A80912C0990912D09FE01E055FD4F44
:104FF000918380830E94560A80914C0990914D09BB
:10500000FE01EE54FD4F918380830E94560A8091E9
:10501000500990915109FE01EC54FD4F918380831A
:105020000E94560A8091540990915509FE01EA5454
:10503000FD4F918380830E94560A8091640990916C
:105040006509FE01E854FD4F918380830E94560A52
:105050008091680990916909FE01E654FD4F9183A2
:1050600080830E94560A80916C0990916D09FE011F
:10507000E454FD4F918380830E94560A8091EC088E
:105080009091ED08A091EE08B091EF08FE01ED556A
:10509000FD4F0197A105B10519F481E0808301C09E
:1050A00010820E94560A8091F0089091F108A09118
:1050B000F208B091F308FE01EC55FD4F0197A105F0
:1050C000B10519F481E0808301C010820E94560A64
:1050D0008091F4089091F508A091F608B091F70836
:1050E000CB55DD4F0197A105B10519F481E0888307
:1050F00001C01882DF91CF911F910F91FF90EF9027
:10510000DF90CF90BF90AF909F908F907F906F90E7
:105110005F904F903F902F9008952F923F924F9223
:105120005F926F927F928F929F92AF92BF92CF9237
:10513000DF92EF92FF920F931F93CF93DF93CDB740
:10514000DEB760970FB6F894DEBF0FBECDBF988B69
:105150008F870E94560AEF85F889E751FE4F81E05C
:1051600040912408509125086091260870912708E5
:10517000452B462B472B09F480E080830E94560A7A
:10518000EF85F889E651FE4F81E040912808509163
:10519000290860912A0870912B08452B462B472B34
:1051A00009F480E080830E94560AEF85F889E55172
:1051B000FE4F81E040912C0850912D0860912E08FF
:1051C00070912F08452B462B472B09F480E08083F4
:1051D0000E94560A8091740890917508A0917608F3
:1051E000B0917708EF85F889E451FE4F8083918371
:1051F000A283B3830E94560A80917808909179081F
:10520000A0917A08B0917B08EF85F889E051FE4FB4
:1052100080839183A283B3830E94560A80917C0885
:1052200090917D08A0917E08B0917F08EF85F88964
:10523000EC50FE4F80839183A283B3830E94560A71
:1052400080914C0890914D08A0914E08B0914F0864
:10525000EF85F889EC5FFD4F80839183A283B38350
:105260000E94560A8091500890915108A0915208CE
:10527000B0915308EF85F889E85FFD4F80839183F3
:10528000A283B3830E94560A8091540890915508D6
:10529000A0915608B0915708EF85F889E45FFD4F5B
:1052A00080839183A283B3830E94560A80915C0815
:1052B00090915D08A0915E08B0915F08EF85F88934
:1052C000E05FFD4F80839183A283B3830E94560ADF
:1052D0008091600890916108A0916208B091630884
:1052E000EF85F889EC5EFD4F80839183A283B383C1
:1052F0000E94560A8091640890916508A091660802
:10530000B0916708EF85F889E85EFD4F808391834F
:10531000A283B3830E94560A8091FC079091FD07F7
:10532000A091FE07B091FF07EF85F889E45EFD4F7D
:1053300080839183A283B3830E94560A80910008E0
:1053400090910108A0910208B0910308EF85F889B7
:10535000E05EFD4F80839183A283B3830E94560A4F
:105360008091040890910508A0910608B091070863
:10537000EF85F889EC5DFD4F80839183A283B38331
:105380000E94560AEF85F889E85DFD4F81E0209183
:10539000D4073091D5072130310509F080E08083B2
:1053A0000E94560AEF85F889E75DFD4F81E0209164
:1053B000D8073091D9072130310509F080E080838A
:1053C0000E94560AEF85F889E65DFD4F81E0209145
:1053D000DC073091DD072130310509F080E0808362
:1053E0000E94560AEF85F889EA5BFD4F81E0409103
:1053F000AC075091AD076091AE077091AF07452B98
:10540000462B472B09F480E080830E94560AEF85E3
:10541000F889E95BFD4F81E04091B0075091B107F9
:105420006091B2077091B307452B462B472B09F4C7
:1054300080E080830E94560AEF85F889E85BFD4F83
:1054400081E04091B4075091B5076091B607709123
:10545000B707452B462B472B09F480E080830E9439
:10546000560AEF85F889E75BFD4F81E0409184089B
:10547000509185086091860870918708452B462BCE
:10548000472B09F480E080830E94560AEF85F88953
:10549000E65BFD4F81E0409188085091890860915A
:1054A0008A0870918B08452B462B472B09F480E026
:1054B00080830E94560AEF85F889E55BFD4F81E005
:1054C00040918C0850918D0860918E0870918F08E2
:1054D000452B462B472B09F480E080830E94560A17
:1054E000EF85F889E45BFD4F81E02091BC073091A6
:1054F000BD072130310509F080E080830E94560A03
:10550000EF85F889E35BFD4F81E02091C007309182
:10551000C1072130310509F080E080830E94560ADE
:10552000EF85F889E25BFD4F81E02091C40730915F
:10553000C5072130310509F080E080830E94560ABA
:105540008091840790918507A0918607B091870785
:10555000EF85F889E15BFD4F80839183A283B3835C
:105560000E94560A8091880790918907A0918A0726
:10557000B0918B07EF85F889ED5AFD4F80839183B9
:10558000A283B3830E94560A80918C0790918D0765
:10559000A0918E07B0918F07EF85F889E95AFD4FEA
:1055A00080839183A283B3830E94560AEF85F88992
:1055B000E65CFD4F81E04091940750919507609122
:1055C000960770919707452B462B472B09F480E0EF
:1055D00080830E94560AEF85F889E55CFD4F81E0E3
:1055E000409198075091990760919A0770919B0795
:1055F000452B462B472B09F480E080830E94560AF6
:10560000EF85F889E45CFD4F81E040919C07509163
:105610009D0760919E0770919F07452B462B472B56
:1056200009F480E080830E94560A80918C09909151
:105630008D09A0918E09B0918F09EF85F889E55DFC
:10564000FD4F80839183A283B3830E94560A809189
:10565000900990919109A0919209B0919309EF85D9
:10566000F889E15DFD4F80839183A283B3830E941B
:10567000560A8091940990919509A0919609B0914C
:105680009709EF85F889ED5CFD4F80839183A283B4
:10569000B3830E94560AEF85F889E35CFD4F81E0F1
:1056A0002091EC073091ED072130310509F080E0C1
:1056B0008083EF85F889E25CFD4F1082EF85F889E1
:1056C000E15CFD4F10820E94560AEF85F889E05C8C
:1056D000FD4F81E02091E8073091E9072130310545
:1056E00009F080E08083EF85F889EF5BFD4F108241
:1056F000EF85F889EE5BFD4F10820E94560AEF8518
:10570000F889ED5BFD4F81E020910C0830910D0888
:105710002130310509F080E080830E94560AEF8530
:10572000F889EC5BFD4F81E0209110083091110861
:105730002130310509F080E080830E94560AEF8510
:10574000F889EB5BFD4F81E020911408309115083A
:105750002130310509F080E080830E94560AEF85F0
:10576000F889E95CFD4F81E020919C0930919D0909
:105770002130310509F080E080830E94560AEF85D0
:10578000F889E85CFD4F81E02091A0093091A109E2
:105790002130310509F080E080830E94560AEF85B0
:1057A000F889E75CFD4F81E02091A4093091A509BB
:1057B0002130310509F080E080830E94560A0F8570
:1057C0001889055A1D4F8091340890913508A09191
:1057D0003608B0913708F80180839183A283B383A0
:1057E0000E94560AEF84F888F1EAEF1AFDEFFF0AEB
:1057F0008091380890913908A0913A08B0913B08FF
:10580000F70180839183A283B3830E94560A80911B
:105810003C0890913D08A0913E08B0913F082F852B
:1058200038892D593D4FF90180839183A283B38339
:10583000F8014081518162817381141615061606A4
:10584000170644F041E050E060E070E0408351838F
:1058500062837383F70140815181628173811416E1
:1058600015061606170644F041E050E060E070E0CF
:105870004083518362837383181619061A061B0628
:105880004CF081E090E0A0E0B0E0F90180839183EA
:10589000A283B383D9018D909D90AD90BC90F70108
:1058A000C080D180E280F380D8014D905D906D90F2
:1058B0007C900E944A1BFC0140825182628273826A
:1058C000C482D582E682F78280869186A286B386DC
:1058D000EF85F889E95CFD4FB081B983EF85F889E0
:1058E000E55DFD4F80819181A281B3814F8558890B
:1058F0004D5B5D4FFA01F081FB834F855889445B16
:105900005D4FFA01F081FA834F855889435C5D4F02
:10591000FA01F081FF834F855889405C5D4FFA01A1
:10592000F081F8874F855889475B5D4FFA01F08118
:10593000F9874F8558894A5B5D4FFA01F081FA87F4
:10594000EF85F889E85DFD4F2080EF85F889E75104
:10595000FE4F3080EF85F889E15BFD4F408151813A
:1059600062817381EF85F889E45EFD4F00811181CA
:1059700022813381EF85F889E05FFD4FC080D180BF
:10598000E280F380EF85F889EC5FFD4F80809180A5
:10599000A280B380EF85F889E451FE4F40805180AA
:1059A00062807380EF85F88940A651A662A673A62F
:1059B00084A695A6A6A6B7A6C0AAD1AAE2AAF3AACB
:1059C00004AB15AB26AB37AB40AF51AF62AF73AF93
:1059D00034AE25AE2A8525A3398536A34A8147A34F
:1059E00040E450E060E070E0E05CFF4F40835183B2
:1059F000628373832885EF85F88926AF3F8137AFAF
:105A0000AF014C5B5F4F2B81FA012083EF85F88952
:105A1000EB5BFF4F80839183A283B383EF85F8898B
:105A2000E75BFF4F39813083AF85B88955968D91FB
:105A30009C9156978633910589F48DEF9FE2FD0185
:105A4000E658FF4F918380833296118210828BEF4C
:105A50009FE2369691838083329630C08C339105D5
:105A600089F485EF9FE2EF85F889E658FF4F91832F
:105A70008083EF85F889E458FF4F1182108283EF0D
:105A80009FE212C08E97E1F48DEE9FE2EF85F889D8
:105A9000E658FF4F91838083EF85F889E458FF4FE4
:105AA0001182108287EE9FE2EF85F889EE57FF4F53
:105AB00091838083EF85F889EC57FF4F1182108224
:105AC000EF85F889838D948D4A97D1F489EF9FE211
:105AD000E258FF4F91838083EF85F889E058FF4FAC
:105AE0001182108287EF9FE2EF85F889EA57FF4F16
:105AF00091838083EF85F889E857FF4F11821082E8
:105B0000EF85F889E85CFD4F20812983EF85F889CE
:105B1000E15DFD4F4080518062807380EF85F889A0
:105B2000EC5BFD4F30813B83EF85F889E35BFD4FF4
:105B30009081EF85F889E25CFD4F40814F83EF85CE
:105B4000F889EF5BFD4F50815887EF85F889E65B58
:105B5000FD4F8081EF85F889E95BFD4FA081AA8721
:105B6000EF85F889E75DFD4F2080EF85F889E651E4
:105B7000FE4F3080EF85F889ED5AFD4F208131814D
:105B8000428153812B873C874D875E87EF85F8895B
:105B9000E05EFD4F4081518162817381EF85F8891C
:105BA000EC5EFD4FC080D180E280F380EF85F88904
:105BB000E85FFD4F80809180A280B380EF85F889F7
:105BC000E657FF4F2F85388920513E4FD9010D915F
:105BD0001D912D913C91008F118F228F338F848ED8
:105BE000958EA68EB78EC0A2D1A2E2A2F3A244A344
:105BF00055A366A377A32B853C854D855E8520A79D
:105C000031A742A753A734A625A63A85358B868BA4
:105C1000978B80E490E0A0E0B0E080AB91ABA2ABCA
:105C2000B3AB488546A75F8157A78B8184AB45AA54
:105C300056AA67AA70AE998191AF85819681863305
:105C4000910589F48DEF9FE2AF85B889AC50BF4FC5
:105C50008D939C93AF85B889AA50BF4F1D921C921B
:105C60008BEF9FE226C08C33910589F485EF9FE28C
:105C7000AF85B889AC50BF4F8D939C93AF85B889E1
:105C8000AA50BF4F1D921C9283EF9FE212C08E97C5
:105C9000E1F48DEE9FE2AF85B889AC50BF4F8D9394
:105CA0009C93AF85B889AA50BF4F1D921C9287EE76
:105CB0009FE2AF85B889A450BF4F8D939C93AF8569
:105CC000B889A250BF4F1D921C92838594854A9734
:105CD000D9F489EF9FE2EF85F889E850FF4F91836F
:105CE0008083EF85F889E650FF4F1182108287EF9D
:105CF0009FE2EF85F889F39591838083EF85F8899A
:105D0000EE5FFE4F11821082EF85F889E75CFD4F50
:105D1000A081A9832F8538892D5C3D4FD9018D91B4
:105D20009D910D90BC91A02D8B839C83AD83BE83F0
:105D3000EF85F889EB5BFD4FB081BA83EF85F88979
:105D4000E25BFD4F20812F83EF85F889E15CFD4FF9
:105D500030813887EF85F889EE5BFD4F40814987B8
:105D6000EF85F889E55BFD4F2080EF85F889E85BDA
:105D7000FD4F3080EF85F889E65DFD4F3081EF857E
:105D8000F889E551FE4F2081EF85F889E95AFD4FEA
:105D900080819181A281B381EF85F889EC5DFD4F0F
:105DA0004081518162817381EF85F889E85EFD4F02
:105DB000C080D180E280F380EF85F889E45FFD4FF9
:105DC00080809180A280B3800F8518890C5F1E4F60
:105DD000EF85F889EC50FE4F4080518062807380DF
:105DE000F801408E518E628E738E848E958EA68EB3
:105DF000B78EC0A2D1A2E2A2F3A244A355A366A388
:105E000077A380A791A7A2A7B3A724A735A7358A10
:105E1000268A2F81278B80E490E0A0E0B0E080AB61
:105E200091ABA2ABB3AB298526A7388537A74A81AA
:105E300044AB8B819C81AD81BE8185AB96ABA7AB1A
:105E4000B0AF298121AF858196818633910589F490
:105E50008DEF9FE2EF85F889E259FE4F91838083B1
:105E6000EF85F889E059FE4F118210828BEF9FE297
:105E700026C08C33910589F485EF9FE2EF85F88980
:105E8000E259FE4F91838083EF85F889E059FE4FF8
:105E90001182108283EF9FE212C08E97E1F48DEEA3
:105EA0009FE2EF85F889E259FE4F91838083EF8569
:105EB000F889E059FE4F1182108287EE9FE2EF854C
:105EC000F889EA58FE4F91838083EF85F889E85876
:105ED000FE4F11821082D8011B968D919C911C97C8
:105EE0004A97E1F489EF9FE2EF85F889EE58FE4F7B
:105EF00091838083EF85F889EC58FE4F11821082E0
:105F000087EF9FE2EF85F889E658FE4F9183808303
:105F1000EF85F889E458FE4F11821082EF85F889E9
:105F2000E65CFD4F20818F8598894096222311F0F1
:105F3000ACD101C096D1EF85F889E55CFD4F208199
:105F40008F85988986579F4F222311F09ED101C0DB
:105F500088D1EF85F889E45CFD4F80818823D1F0FA
:105F6000C80160960FB6F894DEBF0FBECDBFDF91BB
:105F7000CF911F910F91FF90EF90DF90CF90BF9046
:105F8000AF909F908F907F906F905F904F903F90D9
:105F90002F907BC1C80160960FB6F894DEBF0FBE8C
:105FA000CDBFDF91CF911F910F91FF90EF90DF90C8
:105FB000CF90BF90AF909F908F907F906F905F90A9
:105FC0004F903F902F904DC18FEF9FEF0895EBE0E2
:105FD000F1E08081877F80830895EBE0F1E08081AC
:105FE0008860808308958E9808958E9A08951498F5
:105FF0000895149A089588980895889A08950C949D
:10600000D7480C94D7480C94D7480C94D7480C9494
:10601000D7480F931F93CF93DF93FB01C2A1D3A166
:10602000068D178D8091A90B9091AA0B892B41F4B5
:1060300081E090E00E9442489093AA0B8093A90BC4
:106040000430110539F00530110549F4BE0184EE24
:106050009CE003C0BE0181EE9CE00E94CF2380E063
:1060600090E0DF91CF911F910F9108958F929F92B1
:10607000AF92BF92CF92DF92EF92FF920F931F9356
:106080000E94C8191F921F9221E02F931F921F9206
:10609000812C912CA12CB12CC12CD12C76019701F3
:1060A0008601B701A6010E94120D0F900F900F906C
:1060B0000F900F9080E090E01F910F91FF90EF9074
:1060C000DF90CF90BF90AF909F908F9008950E94E7
:1060D0004A1B0E94A71A80E090E0089560E0FC014E
:1060E00083850C94062260E0FC0185810C940622D5
:1060F00061E0FC0183850C94062261E0FC0185814E
:106100000C940622CF93DF93FB01C68DD78D0E949E
:10611000560ABE010E94130A80E090E0DF91CF9101
:10612000089508950895089508951F920F920FB647
:106130000F9211240BB60F922F933F934F935F93BF
:106140006F937F938F939F93AF93BF93EF93FF933F
:10615000E0914407F09145071995FF91EF91BF91A8
:10616000AF919F918F917F916F915F914F913F91EF
:106170002F910F900BBE0F900FBE0F901F90189590
:10618000CF93DF93EC01FC01E759FF4F1082379763
:1061900081E0808360E08D810E9406228F8598894E
:1061A000892B31F060E08B85DF91CF910C94062232
:1061B000DF91CF910895CF93DF93EC018B890E94FB
:1061C000DE212E8930E08217930711F48F8901C0F8
:1061D00080E0DF91CF910895CF93DF93EC0189891F
:1061E0000E94DE212E8930E08217930711F48F89F7
:1061F00001C080E0DF91CF910895CF93DF93EC0150
:106200008DA5882311F061E001C060E08F810E94BC
:1062100006228EA5882329F08FA5882311F061E03E
:1062200001C060E08D85DF91CF910C940622CF9361
:10623000DF93EC018DA5882311F060E001C061E0DF
:106240008F810E9406228EA5882329F08FA588239E
:1062500011F060E001C061E08D85DF91CF910C9479
:106260000622CF93DF93EC0161E089850E9406222C
:106270008EA5882321F061E08F850E940622C959EE
:10628000DF4F1882DF91CF910895CF93DF93EC0118
:1062900060E089850E9406228EA5882321F060E0B7
:1062A0008F850E940622C959DF4F81E08883DF91E4
:1062B000CF910895CF92DF92EF92FF920F931F93A9
:1062C000CF93DF93FC0142AF53AF64AF75AFDC01F6
:1062D000DE964D935D936D937C93139714960D9377
:1062E0001D932D933C931397EC01CA5BDF4FE8821B
:1062F00084A9882389F084A5811109C037FF0CC0C7
:106300001D921D921D921C92139781E006C01016DB
:10631000110612061306A4F380E045A956A967A941
:1063200070AD14161506160617063CF591AD9923A7
:1063300021F10D911D912D913C91139768017901E7
:1063400037FF07C0CC24DD247601C01AD10AE20A47
:10635000F30A4C155D056E057F057CF437FF07C019
:1063600070956095509541955F4F6F4F7F4F4D935E
:106370005D936D937C93139781E0DF01A15BBF4F29
:106380001D921D921D921C921397E15AFF4F91E0AE
:106390009083DF91CF911F910F91FF90EF90DF904D
:1063A000CF9008950F931F93CF93DF938C01D62F37
:1063B000FC018589811109C0C8010EDFC82FC80101
:1063C000FADED11108C08C2F06C0C801F4DEC82F38
:1063D000C80102DFF6CFDF91CF911F910F91089591
:1063E000CF93DF93EC01FC01E759FF4F81E08083FD
:1063F00039978081B297882341F080819181A28171
:10640000B3810196A11DB11D07C080819181A28138
:10641000B3810197A109B10980839183A283B383DA
:10642000FE01E459FF4F20813181DE01A659BF4FA3
:10643000C9019595879520FD03C0ED91FC910DC094
:10644000FE01E80FF91F0190F081E02D2D913C91A4
:10645000E20FF31F0190F081E02D8C0F9D1F199525
:106460008F859889892B11F1FE01E059FF4F20811A
:106470003181DE01A259BF4FC9019595879520FD55
:1064800003C0ED91FC910DC0FE01E80FF91F0190D2
:10649000F081E02D2D913C91E20FF31F0190F081EE
:1064A000E02D8C0F9D1FDF91CF911994DF91CF913B
:1064B00008958F929F92AF92BF92CF92DF92EF9208
:1064C000FF920F931F93CF93DF93EC01FC01E15BED
:1064D000FF4F60817181828193810E94ED4D6B013C
:1064E0007C0168A979A98AA99BA90E94EF4D9B010B
:1064F000AC0160E074E284E799E40E94DD4F4B0157
:106500005C01FE01E55AFF4F6081718182819381B8
:106510000E94ED4D9B01AC01C501B4010E94DD4F0D
:106520004B015C018E010D5A1F4F20E030E040E02E
:106530005FE30E944E4E9B01AC01C701B6010E9471
:10654000794F0E944A50F80160837183828393835C
:10655000C95ADF4FA5019401C701B6010E94794FC6
:106560000E944A50688379838A839B83DF91CF910D
:106570001F910F91FF90EF90DF90CF90BF90AF9061
:106580009F908F9008950F931F93CF93DF93FC01FB
:10659000E759FF4F20812223B9F07A9700811181BA
:1065A0002281338138964081518162817381041741
:1065B00015072607370710F1EC01E2DDCE01DF9168
:1065C000CF911F910F9175CFFC01E15AFF4F2081B0
:1065D0002223A1F0709700811181228133813496AA
:1065E000408151816281738104171507260737079F
:1065F00028F0DF91CF911F910F91F2CEDF91CF91D3
:106600001F910F9108952F923F924F925F926F9238
:106610007F928F929F92AF92BF92CF92DF92EF9232
:10662000FF920F931F93CF93DF93CDB7DEB762979F
:106630000FB6F894DEBF0FBECDBF8C017C0126E4FF
:10664000E20EF11CD7018C919801205A3F4FF801BE
:10665000EF59FF4F6F01A801425C5F4F4A01149749
:106660001D01882341F0F80184A5D9018C9381E0B4
:10667000F60180832FC0DA014D915D916D917C917F
:10668000F10180819181A281B381BB24B394481729
:1066900059076A077B070CF0B12CF901B08277FF2C
:1066A00007C070956095509541955F4F6F4F7F4F34
:1066B000B7FF07C0B095A095909581959F4FAF4FBC
:1066C000BF4F21E0481759076A077B070CF420E009
:1066D000D6012C93F401408151816281738141156F
:1066E00051056105710559F4F801848D958DA68DCC
:1066F000B78DE55AFF4F80839183A283B383F10165
:1067000080819181A281B381F80142AC53AC64AC29
:1067100075AC9801215A3F4F5901481659066A062F
:106720007B0634F4481759076A077B077CF00AC0D8
:1067300084159505A605B7052CF484179507A607BB
:10674000B70724F0D7018C918823D9F0F501808117
:106750008823B9F0D7018C91811105C0F7018081A0
:1067600081110FC006C060E0C8011CDE8111F6CFA8
:1067700017C0D6016C9181E06827C80113DE882319
:1067800079F0D5011C9260E0C8010CDE882309F481
:10679000B3C1F801FE961082118212821382ACC13D
:1067A000D80194962D913D914D915C9197972983B5
:1067B0003A834B835C8358962D913D914D915C912A
:1067C0005B972D833E834F8358875C962D913D9137
:1067D0004D915C915F9729873A874B875C87F101E0
:1067E00080819181A281B381F801FE96C080D18021
:1067F000E280F380F80142AD53AD64AD75ADED5963
:10680000FF4F1082319610823801F5E66F0E711C31
:10681000F301108298012A593F4FF90110823296F4
:1068200010824C015D01841A950AA60AB70AB7FEC8
:1068300008C0B094A09490948094811C911CA11CD9
:10684000B11C481759076A077B072CF4C41AD50AEC
:10685000E60AF70A04C0C81AD90AEA0AFB0AD501EF
:10686000C401B595A795979587958D879E87AF8726
:10687000B88BD801A859BF4F1D01F7FC05C08C1477
:106880009D04AE04BF044CF4F80100A0F1A1E02D7A
:10689000FA8BE98B81E0D9011BC02D853E854F85A0
:1068A00058892C153D054E055F0508F454C08981B3
:1068B0009A81AB81BC818C159D05AE05BF0564F442
:1068C0002D813E812F5F3F4F3A8B298B81E0D30191
:1068D0008C93F10180839EC0C701B6010E94EF4DE9
:1068E0002B013C0169817A818B819C810E94EF4D53
:1068F0009B01AC01C301B2010E94DD4F2B013C01A1
:106900006D817E818F81988529853A854B855C854F
:10691000621B730B840B950B0E94EF4D9B01AC0126
:10692000C301B2010E944E4E2B013C0169857A855C
:106930008B859C850E94EF4D9B01AC01C301B20188
:106940000E94794F0E9445507A8B698B81E0F80153
:10695000ED59FF4F5CC0D501C40129813A814B81BB
:106960005C81821B930BA40BB50BC816D906EA06F3
:10697000FB065CF42D813E812E5F3F4F3A8B298BC5
:1069800081E0F801EB59FF4F42C0C501B4016C1919
:106990007D098E099F090E94EF4D2B013C01698101
:1069A0007A818B819C810E94EF4D9B01AC01C301D8
:1069B000B2010E94DD4F2B013C016D817E818F81F0
:1069C000988529853A854B855C85621B730B840B02
:1069D000950B0E94EF4D9B01AC01C301B2010E94D7
:1069E0004E4E2B013C0169857A858B859C850E94E2
:1069F000EF4D9B01AC01C301B2010E94794F0E948F
:106A000045507A8B698B81E0F801EC59FF4F808308
:106A1000D1018C93F80184818823B1F00E947923FD
:106A2000D80112964D905C901397052C000C6608C7
:106A30007708DC01CB0184199509A609B709893EBD
:106A40009340A105B10568F4F801E55AFF4F298983
:106A50003A89C901A0E0B0E080839183A283B38327
:106A600092CE0E947923D80113967C936E9312974D
:106A700086E294E090D681E296E08DD660E070E008
:106A8000CB01D5D687E296E086D6C701B601CFD630
:106A90008DE296E080D6C501B401C9D683E396E0C5
:106AA0007AD64AE06D857E858F85988975D68AE38A
:106AB00096E071D669817A818B819C81B8D680E419
:106AC00096E069D669857A858B859C85B0D686E403
:106AD00096E061D66D817E818F819885A8D68CE401
:106AE00096E059D682EA94E056D689899A89C6D624
:106AF0008EE993E050D6A8CF62960FB6F894DEBF29
:106B00000FBECDBFDF91CF911F910F91FF90EF90FE
:106B1000DF90CF90BF90AF909F908F907F906F90BD
:106B20005F904F903F902F9008950F931F93FC011B
:106B3000EA5BFF4F2081211110C03897008111813D
:106B4000228133813496408151816281738104179F
:106B500015072607370744F404C0FC0124A52223A7
:106B600019F01F910F9163CB1F910F9146CBFC0140
:106B70001382128214821682158210861782128660
:106B800011861486138616861586108A1786128A31
:106B9000118A148A138ADC01A15ABF4F1C9212AECB
:106BA00013AE14AE15AE91971D921D921D921C92BC
:106BB000139714961D921D921D921C921397149672
:106BC0001C925A961C9211961C9212961C92119627
:106BD0001C9211961C9211961C9211961C92119661
:106BE0001C9211961C9211968DE790E311969C933E
:106BF0008E93129611961C921E92129688E790E33D
:106C000011969C938E93129611961C921E92129638
:106C100083E790E311969C938E93129611961C92A3
:106C20001E9212968EE690E38D939C93E858FF4F48
:106C300011821082089508956E3471050CF050C0D1
:106C40006B3471050CF08FC06C32710554F56932EC
:106C500071050CF088C06831710594F46F307105CE
:106C60000CF081C06630710544F4623071050CF09F
:106C70007AC0672B09F075C076C06B5071096EC081
:106C8000623271053CF46F3171050CF06CC06951D2
:106C9000710964C0645271096230710508F061C005
:106CA00062C06A3371057CF4673371050CF05BC018
:106CB0006D3271050CF455C0603371050CF453C08E
:106CC000635371094BC0643471053CF46134710540
:106CD0000CF049C06D53710941C0675471093EC041
:106CE00066387105F4F463387105ECF562377105A7
:106CF00064F46F367105BCF56536710594F168363C
:106D000071058CF16956710929C06C37710534F42D
:106D10006937710544F56357710920C06D577109D2
:106D20001DC0603D71057CF46D3C7105E4F464396F
:106D3000710534F461397105B4F46D5871090EC0F0
:106D4000695C71090BC06A3D710534F4673D7105DA
:106D500054F4635D710902C06D5D710963307105A2
:106D600010F080E0089581E008952F923F924F92B5
:106D70005F926F927F928F929F92AF92BF92CF92CB
:106D8000DF92EF92FF920F931F93CF93DF93CDB7D4
:106D9000DEB7A3970FB6F894DEBF0FBECDBF9BA39F
:106DA0008AA31B010E948D288AA19BA10E94B22662
:106DB0008AA19BA10E947D268AA19BA10E94812677
:106DC00021E022163104C9F132E02316310409F41E
:106DD00066C02114310409F095C0AAA0BBA040E10F
:106DE000A40EB11C8AA19BA182589E4F9E838D83C5
:106DF000EAA1FBA1EA5BFD4F90819D87AAA1BBA1FF
:106E0000A959BD4FB887AF83EAA1FBA1EF56FD4F4B
:106E1000F98BE88B2AA13BA12D553D4F3D8B2C8B47
:106E20004AA15BA14D515E4F5C874B878DE890E096
:106E30009B8B8A8BA5E1B0E062C0AAA0BBA0BAE898
:106E4000AB0EB11CEAA1FBA1E656FE4FFE83ED831B
:106E5000EAA1FBA1E95BFD4F20812D874AA15BA13F
:106E600045595D4F58874F838AA19BA18D569D4FF1
:106E7000998B888BAAA1BBA1AC55BD4FBD8BAC8BA8
:106E8000EAA1FBA1EB51FE4FFC87EB872EE830E037
:106E90003B8B2A8B46E150E05C834B8336C0AAA033
:106EA000BBA05CEFA51A5EEFB50A8AA19BA18A542C
:106EB0009E4F9E838D83EAA1FBA1E85BFD4F9081ED
:106EC0009D87AAA1BBA1A159BD4FB887AF83EAA1F5
:106ED000FBA1EB56FD4FF98BE88B2AA13BA12B556B
:106EE0003D4F3D8B2C8B4AA15BA149515E4F5C8786
:106EF0004B878FE890E09B8B8A8BA7E1B0E0BC8347
:106F0000AB8303C082E596E00AC0C50165D9811153
:106F100004C0C50150D9882369F083EE96E03BD4C4
:106F20000E944A1B81E090E09093470780934607B8
:106F300090E0CEC386E294E02ED481E896E02BD494
:106F4000D5018C9169D489E197E025D48EE993E04D
:106F500022D481E090E0EB85FC859183808341E041
:106F600050E0B5018AA19BA10E94A21BC5018DD949
:106F7000D5019C968C918501005A1F4F882331F0D2
:106F8000C50155D981E0F801808304C0C50135D918
:106F9000D8011C928D819E810E94910CF501FE9674
:106FA0006083718382839383EF81F88510821182DD
:106FB00012821382EAA1FBA1E959FD4F10821182CE
:106FC00012821382EAA1FBA1E559FD4F10821182C2
:106FD00012821382EAA1FBA1E159FD4F10821182B6
:106FE0001282138286E090E0AB85BC858D939C93E2
:106FF00046E050E0B5018AA19BA10E94A21B41E09E
:1070000050E0B5018AA19BA10E94871B412C512C05
:10701000320143948AA19BA1820D931DFC01ED5581
:10702000FD4FFF87EE874101880C991C880C991C45
:10703000C40189569D4F2AA13BA1280F391F3F8BC0
:107040002E8BC101875A9E4F880F991F4AA15BA1C1
:10705000480F591F5B8F4A8FC4018B579D4FAAA1C0
:10706000BBA1A80FB91FBD8FAC8FF401E758FD4F2E
:10707000FF8FEE8F8AA19BA1880D991D9C01205F37
:107080003D4F3A8729878AA19BA10E945B26AE8546
:10709000BF858C918823B1F0A40149595D4FEAA1C5
:1070A000FBA14E0F5F1FCE88DF88EA8CFB8C0C8D16
:1070B0001D8D2E8D3F8D2E0F3F1F6D817E81C50151
:1070C0000E949F258BEA9BE00E94871E18161906D6
:1070D00024F01A82198210E01DC08BEA9BE00E9406
:1070E000651E8F7D85349105A1F78DE095E053D322
:1070F0000E944A1B21E0DC011C962C9384E693E05D
:107100004AD30E944A1B0E94541AE1E0F0E0FA833D
:10711000E98311E0C50160D88111C9C2C5014BD80E
:107120008111C5C21111C3C2A889B9896D917C9121
:10713000072E000C880B990B0E94EF4D9B01AC01B0
:10714000EF81F88560817181828193810E94E94D90
:1071500087FFADC2C50144D9E985FA852081318117
:107160004281538160E573EC80E090E00E941B4F08
:10717000C9010E943623A985BA852D913D914D9173
:107180005C91A3E0B0E00E94374F9B01AC01C301CA
:10719000B2010E941B4F672B682B692B39F480E6E4
:1071A00093E0F9D20E944A1B0E94541AC5010E9422
:1071B000C030A985BA852D913D914D915C9160E5D6
:1071C00073EC80E090E00E941B4FC9010E943623BF
:1071D000BFEF4B1A5B0A6B0A7B0AE981FA81EF2B3E
:1071E00009F451CF21E030E03A83298342E050E0B6
:1071F000B5018AA19BA10E94871B86E294E0CBD2B5
:1072000081E896E0C8D2D5018C9106D388E896E053
:10721000C2D28EE993E0BFD2E981FA81EF2BD1F49B
:107220008BE996E0B8D282EA94E0B5D288ED94E09A
:10723000B2D28B819C8122D382EA94E0ACD28AEDD7
:1072400094E0A9D2FD858F2F90E018D30E944A1BAD
:107250000E94541A8AA19BA10E947D268AA19BA10B
:107260000E94812686E294E096D281E896E093D24D
:10727000D5018C91D1D28FE996E08DD28EE993E041
:107280008AD2EF81F8851082118212821382D50191
:107290009C968C918501005A1F4F882331F0C501BF
:1072A0000E94FD30F801108206C0C5010E9417310E
:1072B00081E0D8018C938D819E810E94910CF50113
:1072C000FE966083718382839383EAA1FBA1E959CF
:1072D000FD4F1082118212821382EAA1FBA1E559AF
:1072E000FD4F1082118212821382EAA1FBA1E159A3
:1072F000FD4F10821182128213828D819E810E9425
:10730000910C6E8B7F8B888F998F412C512C320181
:1073100043948AA19BA1820D931DFC01ED55FD4F65
:10732000FB8FEA8F9101220F331F220F331F3C8303
:107330002B83C90189569D4F4AA15BA1480F591F54
:107340005D8F4C8FC101875A9E4F880F991FAAA14C
:10735000BBA1A80FB91FBF8FAE8FC9018B579D4F1F
:10736000EAA1FBA1E80FF91FF9A3E8A3C9012AA12B
:107370003BA1820F931FAC01405F5D4F5F874E873B
:107380009201215031093A872987490149815A815F
:10739000452B09F0CBC08AA19BA10E945B26AA8D38
:1073A000BB8D8C918823C9F02B813C8127583D4FA0
:1073B000EAA1FBA12E0F3F1F4B815C8149595D4F14
:1073C0004E0F5F1FCC8CDD8CEE8CFF8C08A119A1B9
:1073D0006D817E81C5010E949F258BEA9BE00E9402
:1073E000871E1816190614F010E01DC08BEA9BE0EA
:1073F0000E94651E8F7D85349105B1F78DE095E083
:10740000CAD10E944A1B21E0DC011C962C9384E621
:1074100093E0C1D10E944A1B0E94541AE1E0F0E0BF
:10742000FA83E98311E029853A852A30310538F459
:10743000AF81B8851D921D921D921C921397BD8538
:10744000C501B11140C10E94DB3081116BC0112315
:1074500019F089849A8466C0E889F989608171810C
:10746000072E000C880B990B0E94EF4D9B01AC017D
:10747000AF81B8856D917D918D919C910E94E94D70
:1074800087FFE7CFC5010E94F031EE85FF8520819F
:1074900031814281538160E573EC80E090E00E948D
:1074A0001B4FC9010E943623AE85BF852D913D91AA
:1074B0004D915C91A3E0B0E00E94374F9B01AC017D
:1074C000C301B2010E941B4F672B682B692B91F4FB
:1074D00080E693E060D10E944A1B0E94541A86E223
:1074E00094E059D183EB96E056D1C201C7D18EE921
:1074F00093E051D1C5010E94C030EE85FF85208107
:1075000031814281538160E573EC80E090E00E941C
:107510001B4FC9010E943623FFEF4F1A5F0A6F0A03
:107520007F0A2ECF81EC96E036D104C081E090E056
:107530009A83898386E294E02ED181E896E02BD16C
:10754000D5018C9169D185ED96E025D18EE993E046
:1075500022D18D819E810E94910CEC89FD89EF2BB7
:10756000A1F0DC01CB012E893F89488D598D821B0A
:10757000930BA40BB50BB7FF07C0B095A0959095E2
:1075800081959F4FAF4FBF4F4C0149815A81452B89
:10759000F9F48BE996E0FFD082EA94E0FCD088ED24
:1075A00094E0F9D08A899B8969D182EA94E0F3D08A
:1075B0008AED94E0F0D0B401092C000C880B990BF3
:1075C0000E94EF4D42E05FD10E944A1B0E94541A74
:1075D00085E090E0AB85BC858D939C9345E050E0C1
:1075E000B5018AA19BA10E94A21BC5010E94313155
:1075F0008AA19BA10E947D268AA19BA10E9481262F
:10760000B1E02B163104A9F0E2E02E16310401F1AD
:10761000232861F50E944A1BC401990CAA0BBB0BDD
:1076200080934C0790934D07A0934E07B0934F075C
:107630001DC00E944A1BC401990CAA0BBB0B80936E
:10764000500790935107A0935207B09353070EC071
:107650000E944A1BC401990CAA0BBB0B80935407D0
:1076600090935507A0935607B09357070E944A1B63
:107670000E94A71AAB85BC851D921C9240E050E089
:10768000B5018AA19BA10E94A21B40E050E0B50178
:107690008AA19BA10E94871B0E944A1BE981FA8153
:1076A000F0934707E093460789819A8111C081ECE6
:1076B00096E071D0C5010E94DB30882309F496CD95
:1076C000B1E0BD8793CD0E94EC308111C2CEBFCE18
:1076D000A3960FB6F894DEBF0FBECDBFDF91CF915A
:1076E0001F910F91FF90EF90DF90CF90BF90AF90E0
:1076F0009F908F907F906F905F904F903F902F90D2
:107700000895CF93DF93FC01EA52FE4F40815181EF
:107710004115510559F1EC01C652DE4F28813981DE
:107720008E529E4F24173507C8F4FC018081918149
:10773000009761F0FC01E20FF31F80818A3041F075
:107740008D3029F48EE993E026D002C080E064D029
:107750008881998101969983888308C040E050E030
:1077600060EA73E00E943C2119821882DF91CF9178
:107770000895009769F0FC0101900020E9F7319726
:10778000AF01481B590BBC018BEA9BE00C94271EF0
:1077900080E090E00895EDCF8F929F92AF92BF92DC
:1077A0000F931F93CF93DF93CDB7DEB7A1970FB69B
:1077B000F894DEBF0FBECDBF19A2423008F44AE0F4
:1077C0008E010F5D1F4F842E912CA12CB12CA50191
:1077D00094010E94474FE62FB901CA0101501109D7
:1077E000EA3014F4E05D01C0E95CD801EC93232B8E
:1077F000242B252B61F7C801BCDFA1960FB6F894A6
:10780000DEBF0FBECDBFDF91CF911F910F91BF9013
:10781000AF909F908F900895E091AB0BF091AC0BDF
:107820000190F081E02D682F8BEA9BE01994CF92B4
:10783000DF92EF92FF92CF93DF9397FF17C06B0118
:107840007C018DE2E9DFEC0166277727CB016C191B
:107850007D098E099F094AE09FDF8C0F9D1FDF91F4
:10786000CF91FF90EF90DF90CF9008954AE0DF91A5
:10787000CF91FF90EF90DF90CF908ECFBC01990F0A
:10788000880B990BD4CF4F925F926F927F928F9219
:107890009F92AF92BF92CF92DF92EF92FF926B01D5
:1078A0007C01B42E9B01AC010E947A50882319F010
:1078B00088E397E027C026013701E89477F82FEF97
:1078C0003FEF4FE75FE7C301B2010E947A50811199
:1078D0000DC02FEF3FEF4FE75FE7C301B2010E94FA
:1078E000E94D18161CF48CE397E00CC02FEF3FEF26
:1078F0004FE75FE4C701B6010E94765018167CF48A
:1079000080E497E0FF90EF90DF90CF90BF90AF9032
:107910009F908F907F906F905F904F902ACF2FEF26
:107920003FEF4FE75FECC701B6010E94E94D87FDCD
:10793000E7CF20E030E0A901C701B6010E94E94D80
:1079400087FF08C08DE268DF4C01F7FAF094F7F882
:10795000F09402C0812C912CA12C60E070E080E0BA
:107960009FE3AB1441F020E030E040E251E40E949C
:10797000DD4FA394F6CF9B01AC01C701B6010E9475
:10798000794F2B013C010E944A506B017C010E94FF
:10799000ED4D9B01AC01C301B2010E94784F2B0158
:1079A0003C014AE0C701B601F7DE7C01E80CF91C96
:1079B000BB2021F08EE230DFE80EF91EDB2CDD204B
:1079C00019F120E030E040E251E4C301B2010E942D
:1079D0004E4E2B013C010E944A504B01A12CB12C70
:1079E0004AE0C501B401D8DEE80EF91EC501B401B4
:1079F0000E94ED4D9B01AC01C301B2010E94784F82
:107A00002B013C01DA94DBCFC701FF90EF90DF90B0
:107A1000CF90BF90AF909F908F907F906F905F902E
:107A20004F900895CF93DF93EC01188A198A1A8A30
:107A30001B8A60E086E10E9406228A8D8295807F03
:107A40000E94CB0C61E086E1DF91CF910C9406227D
:107A5000789484B5826084BD84B5816084BD85B529
:107A6000826085BD85B5816085BD80916E00816035
:107A700080936E00109281008091810082608093DB
:107A800081008091810081608093810080918000DD
:107A90008160809380008091B10084608093B10008
:107AA0008091B00081608093B000809191008260ED
:107AB00080939100809191008160809391008091EA
:107AC00090008160809390008091A10082608093FB
:107AD000A1008091A10081608093A1008091A0000D
:107AE00081608093A00080912101826080932101B8
:107AF000809121018160809321018091200181602A
:107B00008093200180917A00846080937A00809134
:107B10007A00826080937A0080917A0081608093FD
:107B20007A0080917A00806880937A001092C10078
:107B300061E08AE10E94FA2261E08BE10E94FA2270
:107B400061E089E10E94FA2261E08FE00E94FA225E
:107B500061E08EE10E94FA2261E08EE00E94FA224A
:107B600062E085E40E94FA2262E084E40E94FA2244
:107B700062E080E10E94FA2262E081E10E94FA2242
:107B800061E080E20E94FA2261E081E20E94FA2232
:107B900061E08FE10E94FA2262E083E40E94FA220F
:107BA00062E082E40E94FA2262E087E10E94FA2207
:107BB00062E088E10E94FA2261E083E20E94FA22F8
:107BC00061E084E20E94FA2261E082E20E94FA22ED
:107BD00062E081E40E94FA2262E080E40E94FA22DC
:107BE00062E08DE10E94FA2262E08CE10E94FA22BA
:107BF00061E088E20E94FA2261E089E20E94FA22B2
:107C000061E085E20E94FA2261E085E20E9406229C
:107C100061E08DE00E94FA2261E089E00E94FA2290
:107C200061E088E00E94FA2261E087E00E94FA2287
:107C300061E08AE00E94FA2261E08CE00E94FA2270
:107C400062E08FE30E94FA2262E08BE30E94FA2254
:107C500061E084E00E94FA2261E085E00E94FA225D
:107C600061E086E00E94FA2261E087E00E94FA2249
:107C700061E089E10E94062261E08EE00E94062216
:107C800061E08FE10E94062261E082E20E9406220A
:107C900084EF91E0909303028093020262E081E31B
:107CA0000E94FA2261E086E10E94FA2261E086E108
:107CB0000E9406228CB58F7D8CBD8CB5837F8CBDD8
:107CC0008CB58C7F8CBD8DB58E7F8DBDCFB7F89474
:107CD0008091DC0A811127C0E6EBF4E08491E0E7B3
:107CE000F4E09491E82FF0E0EE0FFF1FEF5DFB4F03
:107CF000A591B491EC91E92321F461E085E30E9420
:107D0000062261E085E30E94FA228CB580618CBD79
:107D10008CB580648CBD61E084E30E94FA2261E04E
:107D200083E30E94FA228091DC0A8F5F8093DC0A51
:107D3000CFBFE091BB0BF091BC0B82E08083E09160
:107D4000B70BF091B80B1082E091B90BF091BA0B20
:107D5000D0E1D0831092C30BE091BF0BF091C00B28
:107D600086E08083E091BD0BF091BE0B8081806145
:107D70008083E091BD0BF091BE0B80818860808391
:107D8000E091BD0BF091BE0B808180688083E09113
:107D9000BD0BF091BE0B80818F7D808364E670E027
:107DA00080E090E00E9441230E94C8190E9468165A
:107DB0000E94FB1D0E94CB1D0E9479236093810BC2
:107DC0007093820B8093830B9093840B88EC97E0E5
:107DD0009093450780934407C1E0C0936F00D09310
:107DE000810010928000C093DF0A80E092E09093BF
:107DF000DE0A8093DD0A909387008093860081E1FC
:107E0000809381001092810010928500109284006E
:107E10008091DF0A8061809381000E9479236093C2
:107E20007D0B70937E0B80937F0B9093800B0E9451
:107E300079236093850B7093860B8093870B9093C7
:107E4000880B0E9479236093810B7093820B80933F
:107E5000830B9093840B0E94560A80916007909147
:107E60006107A0916207B09163070197A105B10571
:107E700079F40E94560A8091A8079091A907A091D1
:107E8000AA07B091AB070197A105B10509F4D9C7BD
:107E90000E94560A8091600790916107A091620745
:107EA000B09163070197A105B10579F40E94560AC4
:107EB0008091A4079091A507A091A607B091A7076C
:107EC0000197A105B10509F4DAC70E94560A80910D
:107ED000600790916107A0916207B09163070197D5
:107EE000A105B10579F40E94560A8091A0079091EE
:107EF000A107A091A207B091A3070197A105B10521
:107F000009F4DCC782E893E046DC81E8282E82E0B1
:107F1000382E97E7A92E92E0B92E0E94C8190E9428
:107F20005B260E9479236093850B7093860B809368
:107F3000870B9093880B0091810B1091820B2091FD
:107F4000830B3091840B601771078207930748F405
:107F50006093810B7093820B8093830B9093840BBF
:107F60002CC0DC01CB01801B910BA20BB30B883E14
:107F70009340A105B10508F108511C4F2F4F3F4F09
:107F80000093810B1093820B2093830B3093840B0F
:107F90000E94FB1DEC010E940725CE010C960E9459
:107FA0000725CE0148960E940725CE0184960E949F
:107FB0000725CE01C0960E9407258BEA9BE00E9410
:107FC000871E892B09F4C1C50E94792360937D0B1C
:107FD00070937E0B80937F0B9093800B8BEA9BE0DA
:107FE0000E94651E80937C0B982F9F7D953479F0BD
:107FF00020917A0B30917B0BF901E85BF44F808381
:108000002F5F3F4F30937B0B20937A0B06C00E946B
:108010004A1B21E0DC011C962C9380917A0B9091F5
:108020007B0B8133910564F02AE020937C0BFC01EB
:10803000E85BF44F2083019690937B0B80937A0B3F
:1080400080917C0B20917A0B30917B0B8A3039F434
:10805000C9010197A5E1BBE0E8E4FBE004C02233DD
:108060003105B4F772C5AF0148545B404817590752
:108070001CF441914D93F7CFFC01EB5EF44F10825D
:10808000223031050CF45DC583E193E084DB82EAA4
:1080900094E081DB81EA93E07EDB85E19BE07BDBA2
:1080A00081EA93E078DB8EE993E075DB8AE390E088
:1080B000E9D7EC011A821B821C821D821E821F825C
:1080C000188619861A861B861C861D861E861F86A4
:1080D000188A198A1A8A1B8A1C8A1D8A1E8A1F8A74
:1080E000188E198E1A8E1B8E1C8E1D8E1E8E1F8E44
:1080F00018A219A21AA21BA21CA21DA21EA21FA294
:1081000018A619A61AA61BA61CA61DA61EA61FA663
:1081100018AA19AA1AAA1BAA1CAA1DAA1EAA1FAA33
:1081200018AE19AE6AE072E085E19BE00E947249E8
:108130008C01FC0180818654823008F027C163EAFB
:1081400073E0C8010E947A51892B09F4D3C066EA12
:1081500073E0C8010E947A51892B09F4CBC06AEA06
:1081600073E0C8010E947A51892B09F4C6C06DEAF8
:1081700073E0C8010E947A51892B09F4BEC061EBFB
:1081800073E0C8010E947A51892B09F4B9C065EBEC
:1081900073E0C8010E947A51892B09F4B4C069EBDD
:1081A00073E0C8010E947A51892B09F4ACC06CEBD2
:1081B00073E0C8010E947A51892B09F4A7C060ECD2
:1081C00073E0C8010E947A51892B09F4A2C064ECC3
:1081D00073E0C8010E947A51892B09F49DC068ECB4
:1081E00073E0C8010E947A51892B09F498C06CECA5
:1081F00073E0C8010E947A51892B09F493C060EDA5
:1082000073E0C8010E947A51892B09F48EC064ED95
:1082100073E0C8010E947A51892B09F489C068ED86
:1082200073E0C8010E947A51892B09F484C06CED77
:1082300073E0C8010E947A51892B09F47FC060EE77
:1082400073E0C8010E947A51892B09F47AC064EE68
:1082500073E0C8010E947A51892B09F475C068EE59
:1082600073E0C8010E947A51892B09F470C06CEE4A
:1082700073E0C8010E947A51892B09F46BC060EF4A
:1082800073E0C8010E947A51892B09F466C064EF3B
:1082900073E0C8010E947A51892B09F461C068EF2C
:1082A00073E0C8010E947A51892B09F45CC06CEF1D
:1082B00073E0C8010E947A51892B09F457C060E02D
:1082C00074E0C8010E947A51892B09F452C064E01D
:1082D00074E0C8010E947A51892B09F44DC068E00E
:1082E00074E0C8010E947A51892B09F448C08FEFCD
:1082F0009FEF47C080E090E044C081E090E041C043
:108300008CE190E03EC08DE690E03BC08FE690E0CF
:1083100038C080E790E035C081E790E032C082E766
:1083200090E02FC083E790E02CC084E790E029C064
:1083300088E790E026C089E790E023C08AE790E0D4
:1083400020C083E890E01DC084E890E01AC08DE86A
:1083500090E017C08EE890E014C08FE890E011C064
:1083600080E990E00EC081EA90E00BC085EB90E0E0
:1083700008C086EB90E005C087EB90E002C088EB78
:1083800090E09093010280930002BBC08FEF9FEFBB
:108390009093010280930002B8C0D8018C91883577
:1083A00039F4C80101969BD76A837B838C839D83B4
:1083B000F8018081893539F4C801019690D76E8320
:1083C0007F8388879987D8018C918A3539F4C801D1
:1083D000019685D76A877B878C879D87F801808186
:1083E000813449F4C80101967AD70E9445506E87BE
:1083F0007F87888B998BD8018C91823449F4C8018E
:1084000001966DD70E9445506A8B7B8B8C8B9D8B20
:10841000F8018081833449F4C801019660D70E9435
:1084200045506E8B7F8B888F998FD8018C918335C7
:1084300039F4C801019653D76A8F7B8F8C8F9D8F3B
:10844000F8018081803549F4C801019648D70E941F
:1084500045506E8F7F8F88A399A3D8018C91863564
:1084600049F4C80101963BD70E9445506AA37BA3FB
:108470008CA39DA3F8018081873549F4C80101963A
:108480002ED70E9445506EA37FA388A799A7D80135
:108490008C91853449F4C801019621D70E9445503A
:1084A0006AA77BA78CA79DA7F8018081843549F432
:1084B000C801019614D70E9445506EA77FA788ABCC
:1084C00099ABD8018C918D3449F4C801019607D736
:1084D0000E9445506AAB7BAB8CAB9DABF8018081B1
:1084E000813549F4C8010196FAD60E9445506EAB19
:1084F0007FAB88AF99AF6CE074E080E090E0F2D69B
:108500008C010115110509F048CF0E944A1BDC01BE
:108510001C961C910E94560A40906C0750906D0763
:1085200060906E0770906F07CEA8DFA8E8ACF9AC3A
:108530000E944A1BC0924807D0924907E0924A071E
:10854000F0924B07809100029091010282309105D8
:1085500008F4E9C49C012F5631092530310508F48F
:10856000E2C4992493948437910509F0912C112346
:1085700071F08D36910559F09C012857310923304F
:10858000310528F0855B9109039708F0D0C20E945D
:10859000560A8091600790916107A0916207B0919F
:1085A00063070197A105B10529F0992019F08FEF14
:1085B00092E0BFC2209719F48BEF92E0BAC2E0902C
:1085C0000002F0900102BFEFEB16FB06A9F3E114E5
:1085D000F104B9F48091E00A9091E10A892B61F4E9
:1085E00082E090E04FD523E132E0FC01318320832B
:1085F0009093E10A8093E00A0091E00A1091E10A69
:108600006EC0FCE1EF16F104B9F48091E20A90919A
:10861000E30A892B61F482E090E034D52DE132E069
:10862000DC012D933C939093E30A8093E20A00913E
:10863000E20A1091E30A53C0BDE6EB16F104B9F467
:108640008091E40A9091E50A892B61F482E090E040
:1086500019D527E232E0FC01318320839093E50AAB
:108660008093E40A0091E40A1091E50A53C0FFE602
:10867000EF16F104B9F48091E60A9091E70A892B8C
:1086800061F482E090E0FED421E332E0DC012D933E
:108690003C939093E70A8093E60A0091E60A1091D2
:1086A000E70A53C000E010E0B0E7EB16F104B9F4BC
:1086B0008091E80A9091E90A892B61F482E090E0C8
:1086C000E1D42BE332E0FC01318320839093E90A6B
:1086D0008093E80A0091E80A1091E90A6CC0F1E77A
:1086E000EF16F104B9F48091EA0A9091EB0A892B14
:1086F00061F482E090E0C6D425E432E0DC012D9301
:108700003C939093EB0A8093EA0A0091EA0A109155
:10871000EB0A6CC0B2E7EB16F104B9F48091EC0AF5
:108720009091ED0A892B61F482E090E0ABD42FE4C4
:1087300032E0FC01318320839093ED0A8093EC0AB0
:108740000091EC0A1091ED0A6AC0F3E7EF16F1040C
:10875000B9F48091EE0A9091EF0A892B61F482E0DE
:1087600090E090D429E532E0DC012D933C93909386
:10877000EF0A8093EE0A0091EE0A1091EF0A68C0AA
:10878000B4E7EB16F104B9F48091F00A9091F10A84
:10879000892B61F482E090E075D423E632E0FC019D
:1087A000318320839093F10A8093F00A0091F00ABC
:1087B0001091F10A68C0F8E7EF16F104B9F480915E
:1087C000F20A9091F30A892B61F482E090E05AD486
:1087D0002DE632E0DC012D933C939093F30A8093D5
:1087E000F20A0091F20A1091F30A68C0B9E7EB1699
:1087F000F104A9F48091F40A9091F50A892B51F4BF
:1088000082E090E03FD4FC01B182A0829093F50A0F
:108810008093F40A0091F40A1091F50A6AC0FAE70D
:10882000EF16F104A9F48091F60A9091F70A892BCA
:1088300051F482E090E026D4DC012D923C9290939A
:10884000F70A8093F60A0091F60A1091F70A6CC0B5
:10885000BDE8EB16F104B9F48091F80A9091F90A99
:10886000892B61F482E090E00DD42BE832E0FC012A
:10887000318320839093F90A8093F80A0091F80AD3
:108880001091F90A6CC03EE8E316F104B9F4809146
:10889000FA0A9091FB0A892B61F482E090E0F2D30E
:1088A000E5E9F2E0DC01ED93FC939093FB0A809301
:1088B000FA0A0091FA0A1091FB0A6CC0FFE8EF1661
:1088C000F104B9F48091FC0A9091FD0A892B61F4BE
:1088D00082E090E0D7D3EFE9F2E0DC01ED93FC9386
:1088E0009093FD0A8093FC0A0091FC0A1091FD0A06
:1088F0006CC0F0E9EF16F104B9F48091FE0A909192
:10890000FF0A892B61F482E090E0BCD3E9EAF2E04F
:10891000DC01ED93FC939093FF0A8093FE0A009193
:10892000FE0A1091FF0A6CC0F1EAEF16F104B9F4E7
:108930008091000B9091010B892B61F482E090E013
:10894000A1D3E3EBF2E0DC01ED93FC939093010BF8
:108950008093000B0091000B1091010B6BC0F5EBA5
:10896000EF16F104B9F48091020B9091030B892B5F
:1089700061F482E090E086D3EDEBF2E0DC01ED9370
:10898000FC939093030B8093020B0091020B1091C8
:10899000030B50C0F6EBEF16F104B9F48091040B11
:1089A0009091050B892B61F482E090E06BD3E7ECAA
:1089B000F2E0DC01ED93FC939093050B8093040BA4
:1089C0000091040B1091050B35C0F7EBEF16F10485
:1089D000B9F48091060B9091070B892B61F482E02A
:1089E00090E050D3E1EDF2E0DC01ED93FC93909345
:1089F000070B8093060B0091060B1091070B1AC012
:108A0000F8EBEF16F104B1F48091080B9091090B8B
:108A1000892B61F482E090E035D3E5EEF2E0DC01F1
:108A2000ED93FC939093090B8093080B0091080B36
:108A30001091090B0115110589F48BEF92E00E944A
:108A4000CB3B0E944A1B0E94541A80E194E00E9492
:108A5000B93B8EE993E00E94B93B71C087EF92E089
:108A60000E94CB3B0E944A1B0E94541A0E944A1B40
:108A70001092470710924607E12CF12CFFEFEF1AF6
:108A8000FF0A21E0E216F10441F083EF92E00E9438
:108A9000CB3B0E944A1B0E94541AD801ED91FC91D5
:108AA0000480F581E02DBE01C80119950E944A1B82
:108AB000C0904607D09047070E944A1BFC0184855E
:108AC000E114F104D9F281110AC0E414F5043CF474
:108AD000C114D10421F0F2E0CF16D10479F68BEA6B
:108AE0009BE00E94871E181619062CF48BEA9BE067
:108AF0000E94651EF4CFCD2809F4FFC1992009F426
:108B0000FFC10E94560A8091680790916907A09161
:108B10006A07B0916B070197A105B10509F0F0C193
:108B20000E944A1B21E0DC011C962C93E9C183E0E2
:108B300093E00E94CB3B0E944A1B0E94541ACE0134
:108B400036D310927B0B10927A0B8091140B81110B
:108B500070C00E944A1BFC018485882309F469C007
:108B60000E94C819EC01FC01EE53FD4F10824096A3
:108B70000E943131CE0186579F4F0E943131CE0184
:108B80008C5F9E4F0E9431310E94C60B7C018C018C
:108B9000075C1F4FC1E0D0E06801F8E3CF1AD108AD
:108BA000D6018C918823D9F086E294E00E94CB3BD9
:108BB0008AE294E00E94CB3BCE010E943E3C8EE9CB
:108BC00093E00E94CB3B60E08C2F0E94062240E0A5
:108BD00050E0BE01C7010E945A0BF6011082D80175
:108BE0008C918823F9F086E294E00E94CB3B81E4EB
:108BF00094E00E94CB3BCE010E943E3C8EE993E084
:108C00000E94CB3B61E08C2F0E94FA2260E08C2F07
:108C10000E94062241E050E0BE01C7010E945A0BAB
:108C2000F801108221960F5F1F4FC533D10509F05F
:108C3000B3CF0E944A1BDC011C968C918093140BCD
:108C4000C091120BD091130B0E94560AFC01828135
:108C50009381C817D90799F00E94560ADC01129631
:108C60008D919C9113979093130B8093120B0E94FC
:108C7000C8190E9468160E94FB1D0E94CB1D0E940D
:108C8000792360930E0B70930F0B8093100B9093CE
:108C9000110B00917D0B10917E0B20917F0B309179
:108CA000800B601771078207930708F4BDC0AB0102
:108CB000BC01401B510B620B730B8091020290911F
:108CC0000302092E000CAA0BBB0B84179507A607FD
:108CD000B70708F0B3C00E944A1BFC0184858823B3
:108CE00019F08FE093E002C08BE093E00E94CB3B51
:108CF0000E944A1B0E94541A0E94C819EC01FC01F0
:108D0000ED55FD4F8081882341F0CE0182589E4F62
:108D10000E94910C6B017C0107C0FE01E25BFF4FDA
:108D2000C080D180E280F3800E944A1BC0924C0731
:108D3000D0924D07E0924E07F0924F07FE01EC559E
:108D4000FD4F8081882341F0CE0186569E4F0E94C0
:108D5000910C6B017C0107C0FE01E853FF4FC080FE
:108D6000D180E280F3800E944A1BC0925007D092CB
:108D70005107E0925207F0925307FE01EB55FD4F69
:108D80008081882341F0CE018A549E4F0E94910C2D
:108D90006B017C0106C0CE5BDE4FC880D980EA80C3
:108DA000FB800E944A1BC0925407D0925507E09264
:108DB0005607F09257070E944A1B0E94A71A0E946A
:108DC000C8190E942A1C0E944A1B0E948A1D0E94E8
:108DD0004A1B0E94661A0E94560A80916007909171
:108DE0006107A0916207B09163070197A105B105E2
:108DF00041F087E093E00E94CB3B0E944A1B0E9417
:108E0000541A80910A0B90910B0BA0910C0BB0910E
:108E10000D0B0196A11DB11D80930A0B90930B0BB6
:108E2000A0930C0BB0930D0B0E94792360937D0BE4
:108E300070937E0B80937F0B9093800B0E94241F76
:108E40006CC887E594E00E94CB3B0E94C819CF9381
:108E50001F921F921F921F92812C912CA12CB12C3A
:108E6000C12CD12C760197018601B701A6010E9481
:108E7000120D0F900F900F900F900F9009C88FE672
:108E800094E00E94CB3B0E94C8191F9221E02F93CF
:108E90001F921F921F92812C912CA12CB12CC12CBE
:108EA000D12C760197018601B701A6010E94120D0F
:108EB0000F900F900F900F900F9007C887E894E0E5
:108EC0000E94CB3B0E94C8191F921F9221E02F9352
:108ED0001F921F92812C912CA12CB12CC12CD12C32
:108EE000760197018601B701A6010E94120D0F902D
:108EF0000F900F900F900F9005C88FEE92E002C078
:108F00008BEE92E00E94CB3B0E944A1B0E94541AB7
:108F10000E944A1B109248071092490710924A0774
:108F200010924B070CCE111102CE992493942FCBA3
:108F300088E49CE00C9466211092AE0B1092AD0B6D
:108F400088EE93E0A0E0B0E08093AF0B9093B00B7D
:108F5000A093B10BB093B20B8CE693E09093AC0B63
:108F60008093AB0B85EC90E09093B80B8093B70B9C
:108F700084EC90E09093BA0B8093B90B80EC90E076
:108F80009093BC0B8093BB0B81EC90E09093BE0B55
:108F90008093BD0B82EC90E09093C00B8093BF0B4D
:108FA00086EC90E09093C20B8093C10B1092C40B9F
:108FB0001092C50B1092C60B1092C70B82E090E086
:108FC00061D02EE733E0FC013183208390934F0C76
:108FD00080934E0C60EA73E088E49CE00E946B2171
:108FE0008091E00C803320F09FEF9093E10C11C052
:108FF0008093E10C282F30E0F901EE0FFF1F2E0FB8
:109000003F1FF901E05BF34F28EB3BE03283218304
:109010008F5F803390F48093E40C282F30E0F901C7
:10902000EE0FFF1F2E0F3F1FF901E05BF34F28EB00
:109030003BE0328321838F5F03C09FEF9093E40C6A
:109040008093E00C0895EF920F931F93CF93DF93DB
:10905000E80147FD02C034E001C034E1E42F440FD1
:10906000FF0BF7FF03C0F195E195F109E32E022F05
:109070002E2FAE01B3D1CE01DF91CF911F910F9171
:10908000EF900895CF93DF938230910510F482E042
:1090900090E0E091EB0CF091EC0C20E030E0C0E0CF
:1090A000D0E0309711F14081518148175907C0F045
:1090B0004817590761F482819381209719F09B83A7
:1090C0008A832BC09093EC0C8093EB0C26C0211567
:1090D000310519F04217530718F49A01BE01DF0158
:1090E000EF010280F381E02DDCCF2115310509F17C
:1090F000281B390B2430310590F412968D919C91E8
:1091000013976115710521F0FB019383828304C0DD
:109110009093EC0C8093EB0CFD01329644C0FD0162
:10912000E20FF31F81939193225031092D933C93C9
:109130003AC02091E90C3091EA0C232B41F42091A4
:109140000602309107023093EA0C2093E90C20913B
:109150000402309105022115310541F42DB73EB7C7
:109160004091080250910902241B350BE091E90C53
:10917000F091EA0CE217F307A0F42E1B3F0B28171F
:10918000390778F0AC014E5F5F4F2417350748F080
:109190004E0F5F1F5093EA0C4093E90C819391931B
:1091A00002C0E0E0F0E0CF01DF91CF9108950F938E
:1091B0001F93CF93DF93009709F48CC0FC01329783
:1091C000138212820091EB0C1091EC0C0115110529
:1091D00081F420813181820F931F2091E90C30911D
:1091E000EA0C2817390779F5F093EA0CE093E90CBB
:1091F00071C0D80140E050E0AE17BF0750F412969E
:109200002D913C911397AD012115310509F1D9013B
:10921000F3CF9D01DA013383228360817181860F50
:10922000971F8217930769F4EC0128813981260F73
:10923000371F2E5F3F4F318320838A819B81938329
:109240008283452B29F4F093EC0CE093EB0C42C0A5
:109250001396FC93EE931297ED01499159919E015B
:10926000240F351FE217F30771F480819181840F79
:10927000951F029611969C938E93828193811396EB
:109280009C938E931297E0E0F0E0D80112968D91B6
:109290009C911397009719F0F8018C01F6CF8D91EE
:1092A0009C9198012E5F3F4F820F931F2091E90CF4
:1092B0003091EA0C2817390769F4309729F4109295
:1092C000EC0C1092EB0C02C0138212821093EA0C89
:1092D0000093E90CDF91CF911F910F9108956627BC
:1092E000772709C247EE5CE000C0FA01A191B08186
:1092F000009719F41097E1F0CD01DC01CD010D903C
:10930000002011F4C00113C0FB012191222319F0A8
:109310002015D9F7F3CFFB012191201519F41E92E6
:10932000119606C02223C1F70D900020A1F7D001AD
:10933000FA01A193B0830895BB274A3031F49923F1
:1093400022F4BDE2909581959F4F30C0BB272A3013
:1093500051F4992342F4BDE2909580957095619502
:109360007F4F8F4F9F4F01C0BB27FA01A62F621777
:10937000710581059105330B30FB66F0AA27660F56
:10938000771F881F991FAA1FA21710F0A21B6395B1
:109390003850A9F7A05DAA3308F0A95DA19336F76C
:1093A000B111B1931082CA0104C4BB27FB01552738
:1093B000AA27880F991FAA1FA41710F0A41B839532
:1093C0005051B9F7A05DAA3308F0A95DA1930097A9
:1093D00079F7B111B1931192CB01EBC34F925F9228
:1093E0006F927F929F92AF92BF92CF92DF92EF9255
:1093F000FF920F931F93CF93DF93CDB7DEB72997DB
:109400000FB6F894DEBF0FBECDBF6A01122FB02E8B
:109410002BE3201720F0FF24F394F00E02C0BCE3EE
:10942000FB2E0F2D27E0AE014F5F5F4FCAD2AC017C
:109430008981982F9970913031F0E1FC06C0E0FEEF
:1094400006C090E205C09DE203C09BE201C090E02F
:10945000EE2DE07183FF3CC0911102C083E001C09A
:1094600084E0811718F4212F281B01C020E0E111AE
:109470000BC0F601822F30E2882319F0319381501E
:10948000FBCFC20ED11C20E0992329F0D6019C937A
:10949000F60131966F01C6010396E2FE0AC03EE472
:1094A000D6013C9341E411964C93119712963C934C
:1094B00006C03EE6F601308341E641833283FC017B
:1094C000322F40E2332309F442C041933150FACFA6
:1094D00082FF44C0911102C083E001C084E0811783
:1094E00018F4212F281B01C020E0E1110BC0F60168
:1094F000822F30E2882319F031938150FBCFC20EC6
:10950000D11C20E0992329F0D6019C93F6013196D5
:109510006F01C6010396E2FE0BC039E4D6013C930D
:109520003EE411963C93119736E412963C9307C0A3
:1095300039E6F60130833EE6318336E63283FC01BC
:10954000322F40E2332319F041933150FBCFFC011D
:10955000E20FF11D10828EEF9FEFB7C0F1E0911185
:1095600001C0F0E06F2F70E01416150624F49A0184
:109570002F5F3F4F02C021E030E0260F371FBB2096
:1095800029F06B2D70E06F5F7F4F02C060E070E0EC
:10959000260F371F612F70E0261737071CF4121BA8
:1095A000212F01C020E03E2D387159F4D601322F11
:1095B00060E2332319F06D933150FBCFC20ED11C02
:1095C00020E0FF2331F0D6019C93B6016F5F7F4FFF
:1095D0006B01E1110BC0F601922F30E3992319F0D2
:1095E00031939150FBCFC20ED11C20E09F2D940FE0
:1095F0003A81782F7071A72E84FF03C0313309F4AC
:109600009150191624F4993018F098E001C091E0B7
:10961000E42F852F57FF02C0E0E080E06E2F782F07
:10962000E0E0F0E0AEE29A2E3A01691A71082A01F0
:10963000461A570A0B2D10E01195019511096F3F3D
:109640008FEF780729F4D6019C92C60101966C0130
:109650004617570784F0661677066CF47F01E40C12
:10966000F51CA1E0B0E0AC0FBD1FEA0EFB1ED70158
:109670001196BC9002C090E3B92E615071093196E9
:10968000C60101967C016017710724F0D601BC92D7
:109690006C01D5CF6417750741F4363320F43533A8
:1096A00021F4A11002C081E3B82EF601B082F701C7
:1096B000822F90E2882319F091938150FBCFF7011C
:1096C000E20FF11D108280E090E029960FB6F89429
:1096D000DEBF0FBECDBFDF91CF911F910F91FF90E5
:1096E000EF90DF90CF90BF90AF909F907F906F9062
:1096F0005F904F9008956F927F928F929F92AF925A
:10970000BF92CF92DF92EF92FF920F931F93CF936E
:10971000DF93EC017B016115710519F0DB018D937D
:109720009C938E010F5F1F4F7880872D90E021D290
:10973000892B11F0E801F5CFBDE27B1205C00F5F68
:109740001F4F7980C1E008C0EBE27E1204C08E0199
:109750000E5F1F4F7980C0E06801F1E0CF1AD10899
:1097600043E050E064EF72E0C6010BD2892BE9F4CC
:10977000680122E0C20ED11C45E050E06FEE72E0BD
:10978000C601FFD1892B21F4680187E0C80ED11CE6
:10979000E114F10419F0D701CD92DC92C111F9C0A6
:1097A00060E070E080E89FE7FDC043E050E06CEED1
:1097B00072E0C601E6D1892B51F4E114F10409F4F9
:1097C000EDC00E5F1F4FF70111830083E7C06801F2
:1097D00060E070E0CB0100E010E0F601D0EDD70DC5
:1097E000DA3050F52C2F2260622E2C2F2870C2FF09
:1097F00005C0211127C00F5F1F4F24C0222311F085
:1098000001501109A5E0B0E09B01AC0130D34B0140
:109810005C01880C991CAA1CBB1CC501B4016D0F0E
:10982000711D811D911D6839A9E97A078A07A9E18F
:109830009A0740F0C66005C0DE3F51F4C3FD44C046
:10984000C8606C2EBFEFCB1ADB0A7080C62DC5CF67
:109850002D2F2F7D2531C1F540814D3211F4C0618E
:1098600006C04B3221F0319621E030E006C032963E
:10987000D60111964C9122E030E0A0EDA40FAA3061
:1098800018F0E21BF30B20C040E050E04038BCE091
:109890005B075CF49A01220F331F220F331F420F24
:1098A000531F440F551F4A0F511D3196DF01119769
:1098B0002C91A0EDA20FAA3048F3C4FF03C051952C
:1098C00041955109040F151FC1FF07C0E114F104B0
:1098D00021F03197D701ED93FC937FD1C370C33052
:1098E00019F06B017C0106C06B017C01F7FAF09462
:1098F000F7F8F09420E030E0A901C701B60169D182
:10990000882309F443C017FF06C01195019511097A
:10991000CBE0D3E002C0C3E2D3E05E01B8E1AB1A12
:10992000B1084601BE2DAF2D90E2E92EF12C0E15A7
:109930001F057CF0FE012591359145915491B401AC
:109940008B2F9A2FABD14B01B82FA92F0E191F09BE
:10995000EECF2497F594E794CA15DB0541F764012F
:10996000EB2EFA2E8E2D880F8F2D881F8F3F41F002
:1099700020E030E0A901C701B6012BD1811106C05A
:1099800082E290E09093EE0C8093ED0CC701B6015B
:1099900009C060E070E080E89FEF04C060E070E024
:1099A00080EC9FE7DF91CF911F910F91FF90EF9097
:1099B000DF90CF90BF90AF909F908F907F906F90EF
:1099C0000895283008F027E03327DA01990F311D78
:1099D00087FD916000966105710539F432602E5F54
:1099E0003D9330E32A95E1F708959F3F30F08038AA
:1099F0007105610509F03C5F3C5F3D93913008F0D3
:109A00008068911DDF93CF931F930F93FF92EF9286
:109A1000192F987F9695E92F96959695E90FFF2730
:109A2000EF57FC4F99273327EE24FF24A701E701C6
:109A300005900894079428F4360FE71EF81E491F76
:109A4000511D660F771F881F991F0694A1F7059077
:109A5000079428F4E70EF81E491F561FC11D770F03
:109A6000881F991F661F0694A1F70590079428F494
:109A7000F80E491F561FC71FD11D880F991F661F5B
:109A8000771F0694A1F70590079420F4490F561FFD
:109A9000C71FD81F990F661F771F881F0694A9F745
:109AA00084911095177041F0D695C79557954795B5
:109AB000F794E7941A95C1F7E7E2F3E068941590FC
:109AC000159135916591959105907FE27395E11817
:109AD000F10A430B560BC90BD009C0F7E10CF11E7C
:109AE000431F561FC91FD01D7EF4703311F48A9591
:109AF000E6CFE894015030F0080F0AF4002702176F
:109B000008F4202F2395022F7A3328F079E37D93F0
:109B10002A95E9F710C07D932A9589F606949795C2
:109B20006795379517951794E118F10A430B560B73
:109B3000C90BD00998F023957E9173957A3308F07C
:109B400070E37C932013B8F77E9170617D9330F0C1
:109B5000839571E37D9370E32A95E1F71124EF90EB
:109B6000FF900F911F91CF91DF91992787FD9095DD
:109B700008959111F6C0803219F089508550D0F7C0
:109B80000895FB01DC014150504088F08D918134F3
:109B90001CF08B350CF4805E659161341CF06B35E4
:109BA0000CF4605E861B611171F3990B0895881B9C
:109BB000FCCFDC01FC01672F71917723E1F732972D
:109BC00004C07C916D9370836291AE17BF07C8F398
:109BD000089540D008F481E00895E89409C097FB07
:109BE0003EF490958095709561957F4F8F4F9F4F74
:109BF0009923A9F0F92F96E9BB279395F6958795B8
:109C000077956795B795F111F8CFFAF4BB0F11F47A
:109C100060FF1BC06F5F7F4F8F4F9F4F16C0882321
:109C200011F096E911C0772321F09EE8872F762F57
:109C300005C0662371F096E8862F70E060E02AF098
:109C40009A95660F771F881FDAF7880F9695879584
:109C500097F90895990F0008550FAA0BE0E8FEEF59
:109C600016161706E807F907C0F012161306E407E0
:109C7000F50798F0621B730B840B950B39F40A26D9
:109C800061F0232B242B252B21F408950A2609F4B7
:109C9000A140A6958FEF811D811D08950BD07BC03B
:109CA0006CD028F071D018F0952309F05DC062C027
:109CB0001124A5C081D0A0F3959FD1F3950F50E05A
:109CC000551F629FF001729FBB27F00DB11D639F6E
:109CD000AA27F00DB11DAA1F649F6627B00DA11D14
:109CE000661F829F2227B00DA11D621F739FB00DBA
:109CF000A11D621F839FA00D611D221F749F33272A
:109D0000A00D611D231F849F600D211D822F762FC2
:109D10006A2F11249F5750408AF0E1F088234AF0BF
:109D2000EE0FFF1FBB1F661F771F881F915050400B
:109D3000A9F79E3F510570F017C061C05F3FECF37B
:109D4000983EDCF3869577956795B795F795E795F7
:109D50009F5FC1F7FE2B880F911D9695879597F908
:109D6000089599278827089597F99F6780E870E0FC
:109D700060E008959FEF80EC089500240A94161681
:109D8000170618060906089500240A9412161306E9
:109D9000140605060895092E0394000C11F4882377
:109DA00052F0BB0F40F4BF2B11F460FF04C06F5F93
:109DB0007F4F8F4F9F4F089557FD9058440F551F69
:109DC00059F05F3F71F04795880F97FB991F61F03D
:109DD0009F3F79F087950895121613061406551FB4
:109DE000F2CF4695F1DF08C0161617061806991F20
:109DF000F1CF86957105610508940895E894BB2715
:109E000066277727CB0197F90895F999FECF92BD80
:109E100081BDF89A992780B50895262FF999FECF2C
:109E20001FBA92BD81BD20BD0FB6F894FA9AF99A77
:109E30000FBE01960895052E97FB16F400940FD0DF
:109E400057FD05D024D007FC02D046F408C0509539
:109E50004095309521953F4F4F4F5F4F0895909516
:109E60008095709561957F4F8F4F9F4F089531D0AA
:109E7000A59F900DB49F900DA49F800D911D11245E
:109E80000895B7FFF4CFF3DF821B930B0895A1E28F
:109E90001A2EAA1BBB1BFD010DC0AA1FBB1FEE1F64
:109EA000FF1FA217B307E407F50720F0A21BB30BAF
:109EB000E40BF50B661F771F881F991F1A9469F72B
:109EC00060957095809590959B01AC01BD01CF0187
:109ED0000895A29FB001B39FC001A39F700D811D83
:109EE0001124911DB29F700D811D1124911D0895A3
:109EF0005058BB27AA270ED04ECF3FDF30F044DFAB
:109F000020F031F49F3F11F41EF434CF0EF4E095AD
:109F1000E7FB2ACFE92F50DF80F3BA1762077307F8
:109F20008407950718F071F49EF568CF0EF4E0955C
:109F30000B2EBA2FA02D0B01B90190010C01CA0103
:109F4000A0011124FF27591B99F0593F50F4503EAE
:109F500068F11A16F040A22F232F342F4427585FA0
:109F6000F3CF469537952795A795F0405395C9F7B8
:109F70007EF41F16BA0B620B730B840BBAF0915070
:109F8000A1F0FF0FBB1F661F771F881FC2F70EC00F
:109F9000BA0F621F731F841F48F4879577956795E2
:109FA000B795F7959E3F08F0B3CF9395880F08F0CB
:109FB0009927EE0F9795879508950CD0ECCEE4DEA7
:109FC00040F0DBDE30F021F45F3F19F0CDCE5111CF
:109FD00016CFD0CEF1DE98F39923C9F35523B1F310
:109FE000951B550BBB27AA2762177307840738F008
:109FF0009F5F5F4F220F331F441FAA1FA9F333D067
:10A000000E2E3AF0E0E830D091505040E695001C1A
:10A01000CAF729D0FE2F27D0660F771F881FBB1FD6
:10A02000261737074807AB07B0E809F0BB0B802DB0
:10A03000BF01FF2793585F4F2AF09E3F510568F0FC
:10A0400093CEDDCE5F3FECF3983EDCF386957795BB
:10A050006795B795F7959F5FC9F7880F911D9695FE
:10A06000879597F90895E1E0660F771F881FBB1F5A
:10A07000621773078407BA0720F0621B730B840B07
:10A08000BA0BEE1F88F7E095089504D06894B111DB
:10A09000B6CE089599DE88F09F5790F0B92F992792
:10A0A000B751A0F0D1F0660F771F881F991F1AF0E3
:10A0B000BA95C9F712C0B13081F0A0DEB1E00895C1
:10A0C0009DCE672F782F8827B85F39F0B93FCCF342
:10A0D000869577956795B395D9F73EF490958095D9
:10A0E000709561957F4F8F4F9F4F0895B3DD08F4B2
:10A0F0008FEF0895AFDD880B990B0895EE0FFF1FCA
:10A10000881F8BBF0790F691E02D19946F927F9274
:10A110008F929F92AF92BF92CF92DF92EF92FF9277
:10A120000F931F93CF93DF93EC01009789F4CB013A
:10A13000DF91CF911F910F91FF90EF90DF90CF9023
:10A14000BF90AF909F908F907F906F900C944248FB
:10A15000FC01E60FF71F9C0122503109E217F307BB
:10A1600008F4AAC0D9010D911C9111970617170781
:10A17000A8F00530110508F49DC0C80104978617A2
:10A18000970708F497C002501109061B170B01939B
:10A1900011936D937C93CF010AD88CC05B01A01AF8
:10A1A000B10A4C01800E911EA091EB0CB091EC0C09
:10A1B00040E050E0E12CF12C109709F44AC0A815BA
:10A1C000B905D1F56D907C901197630182E0C80EBE
:10A1D000D11CCA14DB0480F1A3014A195B096A018E
:10A1E00082E0C80ED11C1296BC9012971396AC91C7
:10A1F000B5E0CB16D10440F0B282A38351834083F3
:10A20000D9016D937C930AC00E5F1F4FC301800F6D
:10A21000911FF90191838083EB2DFA2FE114F10452
:10A2200031F0D7011396FC93EE93129743C0F0934D
:10A23000EC0CE093EB0C3EC08D919C91119748176C
:10A24000590708F4AC017D0112960D90BC91A02D28
:10A25000B3CF8091E90C9091EA0C88159905E1F44F
:10A2600046175707C8F480910402909105020097A1
:10A2700041F48DB79EB74091080250910902841BAA
:10A28000950BE817F907C0F4F093EA0CE093E90C9A
:10A29000F901718360830EC0CB010E9442487C01AA
:10A2A000009751F0A801BE011CD0CE010E94D748F2
:10A2B000C70104C0CE0102C080E090E0DF91CF91E1
:10A2C0001F910F91FF90EF90DF90CF90BF90AF90D4
:10A2D0009F908F907F906F90089581E090E0F89428
:10A2E00019C0FB01DC0102C001900D9241505040A9
:10A2F000D8F70895FB01DC018D91019080190110C0
:10A30000D9F3990B0895FB01DC0101900D92002017
:10A31000E1F7089512E0C2EAD2E000E005C0802F24
:10A32000FE01ECDE2196011DC33AD10780E008074B
:06A33000B1F7F894FFCF25
:10A33600FFFF88130000EF0C8000200A0D000000CC
:10A34600000000361A6416E11900000000371A668C
:10A3560016DF1C00000000100D2608B207000000E2
:10A3660000933003303630000000009E25DB1F3B93
:10A376002000000000590B12088B08000000008E18
:10A386000C1808A309000000000F0D2408DB0900C3
:10A396000000000625D91F0420000000000C0D1E39
:10A3A60008330B000000001B360730823000000027
:10A3B600008F0C1A08D40A00000000110D0C087159
:10A3C6000C00000000900C1C08470C000000000E5A
:10A3D6000D22085B0C000000008D0C16080C0C000A
:10A3E6000000009130FF2F093000000000570B0ECF
:10A3F60008E50B00000000943005306730000000CF
:10A40600000D0D2008B9070000000092300130E46D
:10A416002F00000000580B10082808523033005255
:10A42600303200523037005230310052303900524B
:10A43600383800523837005238380052303000521F
:10A4460038370052303800362E342E302E47000072
:10A45600523835005238340052313300523132000E
:10A466005231310052373300523732005237310001
:10A4760052313700523136005231350001000000AA
:10A486000100000001000000523035005230360055
:10A49600523034005238370000000000BD1E271E1F
:10A4A600561E031F871E651E791E000000008C0CB9
:10A4B60014085239392041524455494E4F205354BD
:10A4C600415254555020434F4D504C4554450D0A6A
:10A4D600002A00473000473030004731004730310E
:10A4E60000473238004630390046390046313100DF
:10A4F60046313200463133004631340046313500AC
:10A50600463136004632300046323100463232009D
:10A516004633310046333200463431004634320089
:10A52600463433004634340046363100463831006E
:10A53600463832004638330046383400200A0D00CB
:10A546005239392068616E646C6572203D3D204E3B
:10A55600554C4C0D0A0052393900207265736574EA
:10A5660074696E67206469676974616C2070696ECE
:10A576000020726573657474696E6720616E616C24
:10A586006F672070696E0052393920484F4D45205B
:10A596005A204F4E20535441525455500D0A0052E2
:10A5A600393920484F4D452059204F4E20535441AC
:10A5B600525455500D0A0052393920484F4D452006
:10A5C60058204F4E20535441525455500D0A0052B4
:10A5D600383320005239392057696C6C207A6572FD
:10A5E6006F2058005239392057696C6C207A657291
:10A5F6006F2059005239392057696C6C207A657280
:10A606006F205A005232310050005600523939201C
:10A616004572726F723A20696E76616C6964207059
:10A626006172616D657465722069640D0A0052324B
:10A63600300052343100686F6D650D0A00523939A9
:10A6460020656D657267656E63792073746F700D32
:10A656000A00523939206572726F720D0A0052383B
:10A6660032005239392073746F707065640D0A00B8
:10A67600523939206572726F7220002064656163F9
:10A68600746976617465206D6F746F7220582064EA
:10A69600756520746F206D697373656420737465C6
:10A6A6007073002064656163746976617465206DFA
:10A6B6006F746F7220592064756520746F206D6900
:10A6C60073736564207374657073002064656163D9
:10A6D600746976617465206D6F746F72205A206498
:10A6E600756520746F206D69737365642073746576
:10A6F6007073005239392074696D656F757420580E
:10A7060020617869730D0A005239392074696D65C4
:10A716006F7574205920617869730D0A00523939B2
:10A726002074696D656F7574205A20617869730DA0
:10A736000A0020510052383100205841002058426A
:10A74600002059410020594200205A4100205A4217
:10A756000020737461200020637572200020656EEE
:10A766006420002068616C662000206C656E200005
:10A77600206D696E2000206D617820002073706462
:10A7860020005239392043616C6962726174696FC5
:10A796006E206572726F723A20696E76616C6964BA
:10A7A60020617869732073656C65637465640D0A4E
:10A7B60000206178697320002061742073746172CF
:10A7C60074696E6720706F696E74005232330020B0
:10A7D60063616C6962726174696E67206C656E672D
:10A7E600746800207374657020636F756E743A2008
:10A7F60000523939206D6F76656D656E7420646F11
:10A806006E650D0A0020617420656E6420706F69A4
:10A816006E74005239392043616C696272617469E1
:10A826006F6E206572726F723A20656E6420737463
:10A836006F7020616374697665206265666F726504
:10A846002073746172740D0A00206D6F7665207432
:10A856006F20737461727420666F722063616C6915
:10A8660062726174696F6E006E616E00696E660079
:04A876006F76660093
:00000001FF
